:100000000C9407040C9424040C9424040C946906A6
:100010000C9405190C9424040C9424040C942404CA
:100020000C9424040C9424040C9424040C94D322E3
:100030000C9424040C9424040C9424040C942404A0
:100040000C9466220C9424040C94B9260C94172763
:100050000C9424040C9424040C9424040C94240480
:100060000C9424040C942404A30893119C08931169
:10007000AC081C0993119311260933094009A00902
:1000800093114D0993115B09931165096F099A0842
:100090009311931193117909860993095F107010D8
:1000A0008F1070109310A61099109F10BC10C210E2
:1000B000D110E410FD10071112111C1176137913E1
:1000C0007E138113841387138A138D139013931354
:1000D0009613A213A213A213A213A213A213A21384
:1000E000A2139C1399139F13084AD73B3BCE016E72
:1000F00084BCBFFDC12F3D6C74319ABD56833DDA7F
:100100003D00C77F11BED9E4BB4C3E916BAAAABE8D
:10011000000000803F05A84CCDB2D44EB93836A9B6
:10012000020C50B9918688083CA6AAAA2ABE0000F3
:1001300000803F000D0A4772626C20302E39692022
:100140005B27242720666F722068656C705D0D0A3E
:10015000000D0A003D00244E005D0D0A005B302EAC
:1001600039692E32303135303632303A005D0D0A81
:10017000005B544C4F3A005D0D0A002C005B473980
:10018000323A005D0D0A002C003A0033300032385C
:10019000005B47005D0D0A002053002046002054FC
:1001A00000204D3800204D3900204D3500204D34C1
:1001B00000204D3300204D3200204D3100204D30C5
:1001C00000204739340020473933002047393100B7
:1001D000204739300020473230002047323100209C
:1001E0004731390020473138002047313700204758
:1001F000004733382E00473830004733004732007D
:100200004731004730005B00242420287669657759
:10021000204772626C2073657474696E6773290D70
:100220000A24232028766965772023207061726173
:100230006D6574657273290D0A24472028766965F7
:100240007720706172736572207374617465290D13
:100250000A2449202876696577206275696C6420D4
:10026000696E666F290D0A244E202876696577200D
:100270007374617274757020626C6F636B73290D97
:100280000A24783D76616C75652028736176652057
:100290004772626C2073657474696E67290D0A2455
:1002A0004E783D6C696E65202873617665207374A5
:1002B000617274757020626C6F636B290D0A244340
:1002C0002028636865636B2067636F6465206D6FCA
:1002D0006465290D0A245820286B696C6C20616CB8
:1002E00061726D206C6F636B290D0A24482028729F
:1002F000756E20686F6D696E67206379636C652920
:100300000D0A7E20286379636C65207374617274B2
:10031000290D0A2120286665656420686F6C6429B0
:100320000D0A3F202863757272656E7420737461C4
:10033000747573290D0A6374726C2D7820287265A8
:10034000736574204772626C290D0A005D0D0A0006
:10035000526573746F72696E672064656661756C4F
:1003600074730050676D20456E6400436865636B6D
:1003700020446F6F720044697361626C656400456C
:100380006E61626C65640043617574696F6E3A20DA
:10039000556E6C6F636B656400272448277C2724A7
:1003A000582720746F20756E6C6F636B00526573F5
:1003B000657420746F20636F6E74696E7565005B81
:1003C000000D0A00486F6D696E67206661696C00F8
:1003D00050726F6265206661696C0041626F727471
:1003E00020647572696E67206379636C6500536F72
:1003F0006674206C696D69740048617264206C6970
:100400006D697400414C41524D3A20003E0D0A0086
:100410002C4C696D3A002C52583A002C4275663AC1
:10042000002C002C57506F733A002C002C4D506F4D
:10043000733A003C446F6F72003C436865636B0025
:100440003C416C61726D003C486F6D65003C486FCB
:100450006C64003C52756E003C49646C6500290D6B
:100460000A00206D61782074726176656C2C206DB5
:100470006D0020616363656C2C206D6D2F73656367
:100480005E3200206D617820726174652C206D6D84
:100490002F6D696E002C20737465702F6D6D007A5E
:1004A00000790078002028003D0024002028686F93
:1004B0006D696E672070756C6C2D6F66662C206D93
:1004C0006D290D0A002028686F6D696E67206465CC
:1004D000626F756E63652C206D736563290D0A2448
:1004E00032373D002028686F6D696E67207365653F
:1004F0006B2C206D6D2F6D696E290D0A2432363DEF
:10050000002028686F6D696E6720666565642C2021
:100510006D6D2F6D696E290D0A2432353D00290D50
:100520000A2432343D002028686F6D696E672064AC
:10053000697220696E76657274206D61736B3A0022
:100540002028686F6D696E67206379636C652C2065
:10055000626F6F6C290D0A2432333D0020286861D8
:100560007264206C696D6974732C20626F6F6C29E2
:100570000D0A2432323D002028736F6674206C69A6
:100580006D6974732C20626F6F6C290D0A243231EF
:100590003D0020287265706F727420696E63686513
:1005A000732C20626F6F6C290D0A2432303D0020BD
:1005B0002861726320746F6C6572616E63652C20B4
:1005C0006D6D290D0A2431333D0020286A756E6354
:1005D00074696F6E20646576696174696F6E2C2032
:1005E0006D6D290D0A2431323D00290D0A24313167
:1005F0003D002028737461747573207265706F728A
:1006000074206D61736B3A00202870726F626520F0
:1006100070696E20696E766572742C20626F6F6CE3
:10062000290D0A2431303D0020286C696D69742041
:1006300070696E7320696E766572742C20626F6FBC
:100640006C290D0A24363D002028737465702065DE
:100650006E61626C6520696E766572742C20626FC3
:100660006F6C290D0A24353D00290D0A24343D0004
:10067000202864697220706F727420696E766572CA
:1006800074206D61736B3A00290D0A24333D0020FC
:10069000287374657020706F727420696E7665724D
:1006A00074206D61736B3A00202873746570206943
:1006B000646C652064656C61792C206D73656329B9
:1006C0000D0A24323D002028737465702070756C0B
:1006D00073652C2075736563290D0A24313D002450
:1006E000303D005D0D0A003A002C005B5052423A4A
:1006F000000D0A00496E76616C69642067636F645F
:10070000652049443A00556E646566696E656420EB
:1007100066656564207261746500556E73757070EE
:100720006F7274656420636F6D6D616E64004D6FF0
:1007300064616C2067726F75702076696F6C61748C
:10074000696F6E004C696E65206F766572666C6FBE
:100750007700486F6D696E67206E6F7420656E61FB
:10076000626C656400416C61726D206C6F636B003C
:100770004E6F742069646C6500454550524F4D20A2
:1007800072656164206661696C2E205573696E67BD
:100790002064656661756C74730056616C756520C4
:1007A0003C203320757365630053657474696E670C
:1007B0002064697361626C65640056616C756520C4
:1007C0003C203000496E76616C69642073746174FA
:1007D000656D656E7400426164206E756D62657250
:1007E00020666F726D61740045787065637465642E
:1007F00020636F6D6D616E64206C6574746572004A
:100800006572726F723A20006F6B0D0A000011243E
:100810001FBECFEFD8E0DEBFCDBF11E0A0E0B1E05A
:10082000E4E3F7E702C005900D92A230B107D9F7D3
:1008300026E0A2E0B1E001C01D92A13DB207E1F7C0
:100840000E943B2D0C94983B0C940000F999FECF2C
:1008500092BD81BD81E08FBB80B508958CE1E3E05E
:10086000F1E0DF011D928A95E9F71092A904109238
:10087000AA0481E0809302011092C60108952F928C
:100880003F924F925F926F927F928F929F92AF9220
:10089000BF92CF92DF92EF92FF920F931F93CF936D
:1008A000DF93C091AA04C11101C0C2E1C150D0912F
:1008B000C601CD1709F41BC1EC2EF12C29E2C29F11
:1008C0008001112409531E4FF801A588B688C788F6
:1008D000D08C61A172A183A194A19B01AC010E9463
:1008E0003837F80125A136A147A150A50E948F3ABB
:1008F0004B018C019B01AC01B501C6010E942D3852
:1009000087FD02C05401680189E28E9DF0018F9D30
:10091000F00D1124E953FE4FC501D601818B928B56
:10092000A38BB48BC11101C0C2E1C150CD1761F0DE
:1009300029E22E9DC0012F9D900D11249C01295369
:100940003E4F7901D9E233C08091A904D8135EC02B
:100950000E943E195BC0AC2EB12CDA9DC001DB9D1C
:10096000900D1124FC01E953FE4F6F01C11101C02C
:10097000C2E1C1508091A904C81302C00E943E196F
:10098000DA9D8001DB9D100D112409531E4FF801E3
:1009900085889688A788B08CA501940161897289A1
:1009A000838994890E942D38811106C07601809137
:1009B000C601C813D0CF2AC0F80161A172A183A1DA
:1009C00094A19B01AC010E943837F80125A136A102
:1009D00047A150A50E948F3AF701218932894389A6
:1009E00054890E9438372B013C01A50194010E94D3
:1009F0002D38F80187FF05C0418A528A638A748ABC
:100A0000D5CF818A928AA38AB48AD0CFD091C601E9
:100A1000F9E2DF9F8001112409531E4FC1E0CD0F81
:100A2000C23109F4C0E02090AA0489E2382EC21530
:100A300009F45BC0CC2ED12C3C9CC0013D9C900D98
:100A400011249C0129533E4F7901F80141885288B5
:100A500063887488F90181889288A388B488A50185
:100A60009401C301B2010E942D3887FF24C0F80110
:100A700061A172A183A194A19B01AC010E943837AE
:100A8000F80125A136A147A150A50E948F3A9B01EC
:100A9000AC01C301B2010E9438372B013C01A50112
:100AA00094010E942D3887FF06C0F701418A528ABF
:100AB000638A748ADC2F3C9CF0013D9CF00D11246C
:100AC000E953FE4F258936894789508D618972899E
:100AD000838994890E942D38811101C0DC2FCF5F5A
:100AE000C23109F4C0E08701A2CFD093C601DF91E3
:100AF000CF911F910F91FF90EF90DF90CF90BF901B
:100B0000AF909F908F907F906F905F904F903F90AD
:100B10002F900895009741F0EFE9FFE03197F1F74A
:100B200000C000000197F6CF08958F929F92AF9278
:100B3000BF92CF92DF92EF92FF920F931F93CF93CA
:100B40004B017A016C01C40ED51E8C01C0E05B0123
:100B5000A81AB90AC501800F911F0C151D0599F03F
:100B60000E942604C11108C02C2FCC0F330B232F59
:100B7000221F2227221F01C021E0C22FC80FF80127
:100B800081938F01E7CFC4018E0D9F1D0E94260423
:100B900021E030E0C81711F020E030E0C901CF912A
:100BA0001F910F91FF90EF90DF90CF90BF90AF908B
:100BB0009F908F900895F894F999FECF92BD81BDD2
:100BC00081E08FBB80B58627482F082E000C550B7F
:100BD000262F30E024233523232B39F06F3F19F0E3
:100BE00060BD84E006C084E104C0882321F060BDBC
:100BF00084E28FBBF99A789408958F929F92AF9276
:100C0000BF92CF92DF92EF92FF920F931F93CF93F9
:100C10007C014A016B01C40ED51E8B01C0E05C0152
:100C2000A61AB70AC8018A0D9B1D0C151D0599F05F
:100C3000C11108C02C2FCC0F330B232F221F2227CA
:100C4000221F01C021E0F80161918F01C22FC60F60
:100C50000E94DB05E7CF6C2FC701880D991DCF914E
:100C60001F910F91FF90EF90DF90CF90BF90AF90CA
:100C70009F908F900C94DB05439808958091B40663
:100C800084FD26C09FB7F8948091B406806180935C
:100C9000B4069FBF0E9409250E943C068091B206BF
:100CA000982F9C7021F49091B306913089F49FB7EE
:100CB000843029F4F8948091B506806204C0F894D9
:100CC0008091B50688608093B5069FBF0C947C2206
:100CD00008951F920F920FB60F9211242F933F93F6
:100CE0004F935F936F937F938F939F93AF93BF9334
:100CF000EF93FF938091B206813071F08091B50639
:100D000081110AC00E943E069FB7F8948091B506F3
:100D100083608093B5069FBFFF91EF91BF91AF9124
:100D20009F918F917F916F915F914F913F912F9103
:100D30000F900FBE0F901F9018952F923F924F92D9
:100D40005F926F927F928F929F92AF92BF92CF925B
:100D5000DF92EF92FF920F931F93CF93DF93CDB764
:100D6000DEB7E2970FB6F894DEBF0FBECDBF89E3C2
:100D7000E8E7F6E0DF011D928A95E9F78AE0E9EEFF
:100D8000F5E0A9E7B6E001900D928A95E1F71D8E96
:100D900018A21F8EA12CB12C1AA2212C1E8E9924D0
:100DA0009394F5E03F2E412C512CA0EA6A2EA2E448
:100DB0007A2E8D8DE82FF0E0E756FA4F808088205C
:100DC00009F4EBC29FEB980D9A3110F00C94851149
:100DD0008F5F8D8FBE01675E7F4FCE014D960E9463
:100DE0005D27882311F40C948711C98CDA8CEB8C65
:100DF000FC8CC701B6010E94723B0E94B038162FCE
:100E000070E080E090E00E94E1389B01AC01C701F6
:100E1000B6010E94373720E030E048EC52E40E94EF
:100E20008F3A0E94FC3A0E94B038B7E48B1629F042
:100E3000EDE48E1609F42FC16CC1183209F405C116
:100E4000E8F4143160F4113108F0AAC0143009F448
:100E50004BC008F462C01A30D9F10C9493111C31C4
:100E6000B9F128F4163108F4CAC00C9493111E315C
:100E700079F1163209F451C00C9493111D3309F421
:100E8000DEC0A8F4153309F444C040F41B3209F461
:100E9000BFC0113309F4BCC00C9493111C3310F083
:100EA0000C949311165310937F0609E0D1C01C35A2
:100EB00040F41A3508F083C0103509F46DC00C9465
:100EC00093111C3529F01F3508F490C00C94931130
:100ED0006115710511F00C94A311FE8DFF2311F41F
:100EE0000C94B2110C948911909278060AC01F31AB
:100EF00050F41A3009F0B0C021E02E8F82E08093C8
:100F0000780600E0A5C0153311F00C94E611A1E0BD
:100F1000AE8FB7E0B0937806F4CF8E8D81110C942C
:100F2000891192E09E8F123089F028F4112359F034
:100F3000113081F08CC0163281F0103569F1133018
:100F400009F085C007C01092790681C0AE8DA093CC
:100F500079067DC0109379067AC06E317105A1F0D3
:100F600038F46431710511F00C94931184E010C0D1
:100F70006832710561F06233710511F00C949311C0
:100F8000B7E0B093790606C03092790603C086E0D8
:100F90008093790601E06FC0E8E0E093790657C0DE
:100FA000123129F0133131F010927D0606C0909273
:100FB0007D0603C082E080937D0602E049C0611592
:100FC000710549F41A3519F410927C0602C090920A
:100FD0007C0603E050C06A30710511F00C94931147
:100FE0001A3511F40C94931104E045C01D3519F421
:100FF00090927A0602C010927A0605E029C0143158
:1010000019F490927B0602C010927B0606E020C085
:10101000FE8DF1110C948911113331F410927E067A
:1010200008E023E02E8F27C06A30710511F00C9480
:10103000931190927E0608E083E08E8F1CC0672B90
:1010400011F00C9493110AE016C007E001C001E012
:10105000672B89F00C94AE111C3111F00C94E21145
:1010600081E08E8F6115710511F00C94C51183E03C
:101070008093780600E081E090E0002E02C0880FA7
:10108000991F0A94E2F79C012A213B21232BF1F1BD
:1010900085E10C94EF11672B11F00C94AE11163012
:1010A00018F4133058F017C0183010F40C94931142
:1010B0001A3000F11E3159F00C949311123039F0AE
:1010C0001E3129F0111120C0909280061DC082E0CF
:1010D0008093800619C0143029F0153039F09092B1
:1010E000820606C082E08093820602C010928206C9
:1010F0000CE0C1CF193021F082E08093810602C05C
:10110000109281060DE0B7CF0BE0B5CFA82AB92A1F
:1011100050CE882D880C990BAA0BBB0BFC01E15417
:10112000F109EA31F10510F00C949311EC5CFF4FDA
:101130000C94173709E005C1C701B6010E94B03809
:1011400060936B0606C0C701B6010E94B038609379
:101150006C060E947225F5C0C701B6010E94A9382D
:1011600070930101609300016230710581F1A4F474
:101170006130710571F740922806509229066092FD
:101180002A0670922B0640922C0650922D066092F1
:101190002E0670922F064BC06330710579F16430D2
:1011A0007105B9F680E090E0A8ECB3E480932806DE
:1011B00090932906A0932A06B0932B0680932C06C1
:1011C00090932D06A0932E06B0932F0630C080E09A
:1011D00090E0A8ECB2E48093280690932906A093AF
:1011E0002A06B0932B0680932C0690932D06A0938D
:1011F0002E06B0932F0690926B0616C080E090E00A
:10120000A0EAB1E48093280690932906A0932A06C9
:10121000B0932B0680932C0690932D06A0932E0658
:10122000B0932F0610926B0690926C0692CF10929C
:101230006B0610926C068DCFC0928306D092840606
:10124000E0928506F092860600E07BC0C092870699
:10125000D0928806E0928906F0928A069AA191605F
:101260009AA301E06EC0C0928B06D0928C06E092E9
:101270008D06F0928E06AAA1A260AAA302E061C028
:10128000C0928F06D0929006E0929106F09292065C
:10129000BAA1B460BAA303E054C0C701B6010E946A
:1012A000A938609394067093950680939606909360
:1012B000970605E046C0C0929806D0929906E09243
:1012C0009A06F0929B0606E03CC0C0929C06D09223
:1012D0009D06E0929E06F0929F0607E032C0C09203
:1012E000A006D092A106E092A206F092A30608E022
:1012F00028C0C092A506D092A606E092A706F0925A
:10130000A806E22DE1602E2E0AE01BC0C092A906BD
:10131000D092AA06E092AB06F092AC06F22DF260F3
:101320002F2E0BE00EC0C092AD06D092AE06E0921A
:10133000AF06F092B006222D2460222E0CE001C0F0
:1013400004E0EE24E394F12C002E02C0EE0CFF1C0E
:101350000A94E2F78F8D98A18E219F21892B09F0A5
:10136000DAC781E693E0002E02C0959587950A942E
:10137000E2F780FF0BC020E030E0A901698D7A8D93
:101380008B8D9C8D0E942D3887FDC7C78F8D98A1AE
:101390008E299F2998A38F8F0CCD222029F09E8D16
:1013A000911102C0A2E0AE8FBF8DB5FF0EC080913B
:1013B000940690919506A0919606B0919706803874
:1013C0009649A849B1050CF0AAC780917A068130E8
:1013D00039F4FE8DF230B1F52F8D20FFAAC732C04F
:1013E0008091EA0581112EC08F8D80FF1BC08091F6
:1013F0007B06813039F523E333E34BEC51E4609114
:1014000083067091840680918506909186060E94DD
:101410008F3A609383067093840680938506909339
:10142000860610C08091F7059091F805A091F90506
:10143000B091FA058093830690938406A093850665
:10144000B0938606AF8DB8A1B0FD10C08091F305B2
:101450009091F405A091F505B091F6058093A00652
:101460009093A106A093A206B093A306809178065C
:10147000813051F4BF8DB6FD02C08CE1B0C7EF8D55
:10148000F8A1EF7BF8A3EF8F80917D06882371F0A0
:10149000813031F4F1E0F8A71FA222E02EA30BC0A7
:1014A00018A682E08FA391E09EA305C0A2E0A8A7A2
:1014B000B1E0BFA31EA280917B06813021F0EE8DAA
:1014C000E33091F52AC075EAE72E76E0F72E00E0CA
:1014D00010E0C22CD12CC601002E02C09595879534
:1014E0000A94E2F780FF10C023E333E34BEC51E4AE
:1014F000D7016D917D918D919C910E948F3AF7015A
:1015000060837183828393830F5F1F4FF4E0EF0E3C
:10151000F11C03301105F9F6D2CF80917E0681309F
:1015200019F424E02212FDC68CE0ECE0F6E0DE01C6
:101530001D9601900D928A95E1F7B1FC09C080914A
:10154000780689A38230B9F0883009F4B2C012C19C
:1015500080917F06873010F08DE141C79091EF05B3
:10156000981769F3BE01635F7F4F0E948825882327
:1015700009F4E7C6E4CF211002C08AE130C78F8D9D
:1015800098A180759927892B09F477CF60919806E7
:101590007091990680919A0690919B060E94723BE9
:1015A0000E94B0386730C0F680919306843131F0E4
:1015B000823009F0B8C69F8D97FDB5C6AF8DB8A132
:1015C000AF7AB8A3AF8F662319F0615069A303C047
:1015D000B0917F06B9A3BE016F5F7F4F89A10E94C2
:1015E0008825882309F4ADC63090930640902406E0
:1015F0005090250660902606709027068E010F5F9A
:101600001F4FC12CD12CE12CF12C822C912CC40128
:101610000E2C02C0959587950A94E2F780FF3BC097
:10162000F601E858F94F5F01F4E13F122AC0F601D4
:10163000E751FA4F27A530A941A952A96789708DB2
:10164000818D928D0E943737D5019D962D913D91C8
:101650004D915C91D0970E943737F8016083718378
:1016600082839383F2E0EF16F104A9F4A3019201BF
:101670000E943737D8016D937D938D939C93139778
:101680000AC0F50185A596A5A7A5B0A9F801808394
:101690009183A283B383FFEFEF1AFF0A24E0C20E07
:1016A000D11C0C5F1F4F83E0E816F10409F0AFCFA7
:1016B0000FC1222009F461CF4090240650902506E6
:1016C000609026067090270605EA16E0C12CD12C02
:1016D000E12CF12CA22CB12CF601E751FA4FC501F7
:1016E0000E2C02C0959587950A94E2F780FF2BC0D7
:1016F000ADE0B0E0AC0FBD1FAC0DBD1D2D913D9117
:101700004D915C916789708D818D928D0E943737E4
:10171000D8012D913D914D915C910E943737F80190
:101720006083718382839383F2E0EF16F104A1F466
:10173000A30192010E943737D8016D937D938D9359
:101740009C93139709C087A590A9A1A9B2A9F801F4
:1017500080839183A283B383FFEFEF1AFF0A24E013
:10176000C20ED11C0C5F1F4F83E0E816F10409F094
:10177000B3CFADC09E8D933059F4A9A1A53009F423
:101780008EC0A73009F49EC0A33009F0A0C07FC06E
:10179000222009F491C030907C064090240650909D
:1017A0002506609026067090270660E0C62E66E04B
:1017B000D62E05EA16E05E01BDE0AB0EB11CE12CB1
:1017C000F12C822C912CC4010E2C02C0959587958A
:1017D0000A94E2F780FD0BC0F60180819181A2811D
:1017E000B381F80180839183A283B3833FC0F9A1C1
:1017F000F730E1F1311029C0D60158962D913D9175
:101800004D915C915B97F50160817181828193813B
:101810000E943837D8012D913D914D915C910E94E5
:101820003837F8016083718382839383F2E0EF1687
:10183000F104E1F4A30192010E943837D8016D93BD
:101840007D938D939C93139711C0F6012081318174
:1018500042815381D8016D917D918D919C910E941F
:101860003837F8016083718382839383FFEFEF1A27
:10187000FF0A24E0C20ED11C0C5F1F4F84E0A80EAB
:10188000B11C93E0E916F10409F09DCF76CF211049
:1018900001C01E8EBE016F5F7F4F86E007C0211022
:1018A00001C01E8EBE016F5F7F4F87E00E948825BA
:1018B000882309F446C50BC0E9A1E53091F3E73070
:1018C00009F089C580917906823008F02EC519A2E9
:1018D00010917906183041F4222009F4DEC1AE8D52
:1018E000A13009F024C5BDC2BE8DB23009F0D5C10A
:1018F0001123D9F020E030E0A901609183067091B6
:10190000840680918506909186060E942D38882352
:1019100009F40FC5143028F4123058F4113029F0AE
:10192000A0C2183008F478C19CC2222009F4B8C1C2
:1019300098C2222009F421CEEEA16E2E712C9FA117
:10194000892F90E09AA789A781E090E07C010FA001
:1019500002C0EE0CFF1C0A94E2F702C0880F991F28
:10196000EA95E2F7E82AF92A822D90E08E219F215C
:10197000892B09F4E0C4C301880F991F880F991FB0
:10198000FC01E858F94FDC01A751BA4F57962D9149
:101990003D914D915C915A9765A576A587A590A933
:1019A0000E9437371B012C0189A59AA5880F991F22
:1019B000880F991FFC01E858F94FDC01A751BA4F75
:1019C00057962D913D914D915C915A9765A576A5BD
:1019D00087A590A90E9437374B015C01CF8CD8A016
:1019E000A0E8CA22DD24BF8DB7FF43C0EF8DF8A168
:1019F000EF77F8A3EF8F2091A5063091A6064091CE
:101A0000A7065091A806609100067091010680918A
:101A10000206909103060E942D38811147C1209142
:101A2000A9063091AA064091AB065091AC06609190
:101A300004067091050680910606909107060E94A3
:101A40002D38811133C12091AD063091AE06409101
:101A5000AF065091B006609108067091090680911A
:101A60000A0690910B060E942D3881111FC181E258
:101A7000B6C49AA1892F90E09BA38AA3E822F922F9
:101A8000EF2809F45AC4AF8DB8A1A17FB8A3AF8FD6
:101A900080917B06813009F47AC0F301EE0FFF1FBD
:101AA000EE0FFF1FE458F94FC384D484E584F68415
:101AB000A7019601C201B1010E9437372B013C01F9
:101AC000E9A5FAA5EE0FFF1FEE0FFF1FE458F94F2F
:101AD00083859485A585B6858AA39BA3ACA3BDA366
:101AE0009C01AD01C501B4010E9437374B015C0177
:101AF000A3019201C301B2010E948F3A2B013C0164
:101B0000A5019401C501B4010E948F3A9B01AC016B
:101B1000C301B2010E9438370E942E3B4B015C0189
:101B2000A7019601C701B6010E948F3A6B017C01A3
:101B30002AA13BA14CA15DA1CA01B9010E948F3A23
:101B40009B01AC01C701B6010E9438370E942E3BB1
:101B50006B017C0160939C0670939D0680939E06AA
:101B600090939F069B01AC01C501B4010E943737D9
:101B70004B015C01E894B7F82AE037ED43EA5BE3F8
:101B8000C501B4010E944F3A18164CF16AC108E72A
:101B900016E08AA19BA10C2C02C0959587950A940A
:101BA000E2F780FF12C023E333E34BEC51E4D801AA
:101BB0001F966D917D918D919C9152970E948F3AC5
:101BC000F8016787708B818B928BFFEFCF1ADF0A4A
:101BD0000C5F1F4F23E0C216D104D9F65ECF20E080
:101BE00030E040E05FE3C501B4010E944F3A1816AF
:101BF0000CF43DCF2FE632E143E85AE3C701B601CA
:101C00000E948F3A9B01AC01C501B4010E944F3A7A
:101C100018160CF42CCF25C1222009F4AECC20914B
:101C2000A5063091A6064091A7065091A80660919E
:101C300000067091010680910206909103060E94B1
:101C40002D3881110EC12091A9063091AA0640912C
:101C5000AB065091AC066091040670910506809128
:101C60000606909107060E942D388111FAC0209136
:101C7000AD063091AE064091AF065091B00660912E
:101C800008067091090680910A0690910B060E9441
:101C90002D38882309F4EBCEE4C08E8D8111E1C08C
:101CA0008F8D98A18E7D9C7F1E8EDFC080917B06DC
:101CB0008130B1F423E333E34BEC51E460919C06B3
:101CC00070919D0680919E0690919F060E948F3A8A
:101CD00060939C0670939D0680939E0690939F064A
:101CE00080919C0690919D06A0919E06B0919F06C2
:101CF0008AA39BA3ACA3BDA3A2019101C201B10120
:101D00000E948F3A6BA77CA78DA79EA7A50194017F
:101D1000C501B4010E948F3A6FA778AB89AB9AAB2B
:101D200020E030E040E850E46AA17BA18CA19DA1B5
:101D30000E948F3A2AA13BA14CA15DA10E948F3A3B
:101D40002BA53CA54DA55EA50E9437372FA538A928
:101D500049A95AA90E9437376B017C0120E030E085
:101D6000A9010E942D3887FDFBC2C701B6010E9460
:101D70002E3B6B017C012FA538A949A95AA96BA557
:101D80007CA58DA59EA50E9438370E942E3B9B0105
:101D9000AC01C701B60190580E9437386B017C0135
:101DA000133021F4F7FAF094F7F8F09420E030E0E3
:101DB000A9016AA17BA18CA19DA10E942D3887FF5A
:101DC00011C0F7FAF094F7F8F0948AA19BA1ACA1A6
:101DD000BDA1B05880939C0690939D06A0939E064B
:101DE000B0939F068301000F111F000F111F0458AD
:101DF000194FA7019601C501B4010E948F3A9B01BA
:101E0000AC01C201B1010E94373720E030E040E070
:101E10005FE30E948F3AD8011B966D937D938D935B
:101E20009C931E9709A51AA5000F111F000F111FE3
:101E30000458194FA7019601C201B1010E948F3ABF
:101E40009B01AC01C501B4010E94383720E030E0AD
:101E500040E05FE30E948F3AF801638774878587CB
:101E600096878F8D98A18E7D907E892B09F067C211
:101E70008091940690919506A0919606B091970650
:101E80008093FC059093FD05A093FE05B093FF059C
:101E900080917A068093EA0580918306909184066A
:101EA000A0918506B09186068093F7059093F8057A
:101EB000A093F905B093FA05C090A006D090A106B2
:101EC000E090A206F090A306A70196016091F305A9
:101ED0007091F4058091F5059091F6050E942D38DA
:101EE0008823C1F08091F205882321F0B701A60173
:101EF0000E94C3328091A0069091A106A091A206F3
:101F0000B091A3068093F3059093F405A093F50593
:101F1000B093F6058091A4068093FB05809182061C
:101F20009091F205981771F04091F3055091F405E6
:101F30006091F5057091F6050E94C332809182068A
:101F40008093F205109181068091F105811781F04F
:101F50008091B206823041F00E94A632123011F414
:101F6000439A02C00E943C06809181068093F1054D
:101F700080917806813069F080917D068093ED052F
:101F800080917B068093EB059E8D933009F074C0A1
:101F900054C08090980690909906A0909A06B090B0
:101FA0009B068091B206823039F320E030E040EAAF
:101FB00051E4C501B4010E948F3A0E941C390E946D
:101FC000B0386B017C010E94A63220E030E04AE785
:101FD00054E4C501B4010E948F3A4B015C0182E3D5
:101FE0008C9DB0018D9D700D112480E090E00E94C9
:101FF000DF389B01AC01C501B4010E9437370E9454
:102000001C390E94B038CB010E948A05C114D1044A
:1020100009F4B2CF0E943D15A1E0CA1AD1088091FF
:10202000B1068111A9CFBFEFE0E7F2E0B150E04087
:10203000F040E1F700C00000E9CF80917E06809378
:10204000EE05813089F48091AD069091AE06A091A5
:10205000AF06B091B0068093240690932506A09316
:102060002606B093270608C0109224061092250673
:10207000109226061092270680917F069091EF0518
:10208000981759F08093EF058CE0FE013D96ACE087
:10209000B6E001900D928A95E1F780917C068093DD
:1020A000EC05E09178068E2F90E0FC013297E83045
:1020B000F10508F04BC0E25BFF4F0C941737BE01EF
:1020C0006F5F7F4F89A10E947F258091EF0529A135
:1020D00082133CC08CE0FE013196ACE0B6E01AC041
:1020E0008E8D882349F020E040E050E060E87FEBEF
:1020F00085EA96E00E940E2820E040E050E060E88B
:102100007FEBCE0101960E940E288CE0FE013196F5
:10211000A0E0B6E001900D928A95E1F717C060E06B
:1021200076E086E003C060E076E087E00E947F25ED
:102130000DC08CE0E5EAF6E0A8E1B6E0EBCF8CE07C
:10214000E8E1F6E0DF011D928A95E9F7E091790672
:10215000E093E905E83009F486C0BE8DB23009F09D
:1021600082C08E2F90E08830910508F073C0FC018A
:10217000EA5AFF4F0C94173720E040E050E060E847
:102180007FEB0AC04091F7055091F8056091F90581
:102190007091FA052091EA0585EA96E00E940E28E2
:1021A00059C02091F7053091F8054091F9055091FB
:1021B000FA0560919C0670919D0680919E06909113
:1021C0009F068824839411C02091F7053091F8056B
:1021D0004091F9055091FA0560919C0670919D0619
:1021E00080919E0690919F06812CA8A4CFA0EEA07E
:1021F0000091EA050E94EB332DC06091F7057091C4
:10220000F8058091F9059091FA0500E009C0609108
:10221000F7057091F8058091F9059091FA0501E0B4
:1022200020E014C06091F7057091F8058091F905E0
:102230009091FA0500E009C06091F7057091F805EA
:102240008091F9059091FA0501E021E04091EA05BD
:102250000E9441338CE0E5EAF6E0A0E0B6E00190B0
:102260000D928A95E1F7809180068093F00588238E
:1022700009F4B5C00E94A6329091F0058091B20693
:10228000913069F48230E9F19FB7F8948091B406F7
:1022900088608093B4069FBF0E943D1532C091E0D4
:1022A0009093E9051092ED051092EC051092EA0565
:1022B0001092EF051092F2051092F1058230A9F00C
:1022C000BE01635F7F4F80E00E9488258823C9F1AB
:1022D0008CE0FE013D96ACE0B6E001900D928A954F
:1022E000E1F70E9409250E943C068FEB93E00E94D3
:1022F000561383E693E00E9456138CE493E00E9409
:1023000056131092F00580E06AC081E068C082E058
:1023100066C088E164C089E162C084E060C08BE18E
:102320005EC085E25CC084E15AC08EE158C08FE196
:1023300056C086E154C080E252C083E250C084E2BD
:102340004EC087E04CC01E3199F028F51A3011F4C8
:102350000C947E071C3111F40C94320887E13FC0C5
:1023600082E23DC01E3111F00C94770791E09E8F00
:102370006115710531F06A307105A9F686E00C949B
:102380003808309278060C943A086A30710559F68C
:1023900084E00C943808153311F40C9489071C352B
:1023A000E9F66115710549F06A30710509F0BBCF96
:1023B00029E0209378060C943A08F8E0F093780628
:1023C0000C943A0891E09E8F0C943A081C35D1F792
:1023D000E1E0EE8FE6CFE33009F079CA5ACAE2961F
:1023E0000FB6F894DEBF0FBECDBFDF91CF911F9126
:1023F0000F91FF90EF90DF90CF90BF90AF909F90A4
:102400008F907F906F905F904F903F902F900895A6
:10241000CF93DF93C9E9D5E08991882319F00E9411
:102420004127FACFDF91CF910895CF93DF9321E534
:10243000829FC0011124EC01DD5F40E550E0BE0148
:1024400089E995E00E949505892B59F41092990528
:1024500040E550E069E975E0CE010E94FD0580E0AD
:1024600001C081E0DF91CF9108958F929F92AF924A
:10247000BF92CF92DF92EF92FF920F931F93CF9371
:10248000DF93CDB7DEB72A970FB6F894DEBF0FBE45
:10249000CDBF6B017C01042F20E030E0A9010E9438
:1024A0002D3887FF07C08DE20E944127F7FAF0948C
:1024B000F7F8F094102F123060F020E030E048EC94
:1024C00052E4C701B6010E948F3A6B017C011250A1
:1024D000F2CF00FF0AC020E030E040E251E4C70143
:1024E000B6010E948F3A6B017C0120E030E040E0B1
:1024F0005FE3C701B6010E9438370E94A938E1E0C6
:10250000F0E0EC0FFD1FE00FF11D2EE2208310E044
:102510003AE0832E912CA12CB12C61157105810517
:102520009105A9F0101301C01F5FEE24E394F12C74
:10253000EC0EFD1EE10EF11CA50194010E94D636A1
:10254000605DF7016083B901CA011F5FE6CF80E3D8
:10255000101748F4E1E0F0E0EC0FFD1FE10FF11D72
:1025600080831F5FF5CF10130BC012E0100F0F5FB9
:10257000E1E0F0E0EC0FFD1FE00FF11D80E3808350
:10258000112341F0FE01E10FF11D80810E944127DE
:102590001150F6CF2A960FB6F894DEBF0FBECDBF0E
:1025A000DF91CF911F910F91FF90EF90DF90CF902F
:1025B000BF90AF909F908F90089543E00C94351298
:1025C000EF92FF920F931F93CF93DF931F92CDB79C
:1025D000DEB7362FEDB6FEB66DB77EB7641B710958
:1025E0000FB6F8947EBF0FBE6DBF0DB71EB70F5F5D
:1025F0001F4F202FF8019E2F921B941728F4632F52
:102600000E94CA369193F7CF442361F0F801E40F9A
:10261000F11D31978081805D49830E944127498166
:102620004150F2CF0FB6F894FEBE0FBEEDBE0F9034
:10263000DF91CF911F910F91FF90EF90089548E0A7
:1026400062E00C94E0129FB7F894E1EBF6E083812E
:10265000826083839FBF08952091650620FF08C094
:102660002BE832E441E25DE30E948F3A41E001C091
:1026700040E00C9435122091650620FF08C02BE83D
:1026800032E441E25DE30E948F3A44E001C043E05E
:102690000C9435128A3020F0843620F043E003C0D9
:1026A00041E001C042E06AE00C94E012CF93DF9376
:1026B000FC018491EF012196882321F00E9441279B
:1026C000FE01F7CFDF91CF910895CF93C82F80E01F
:1026D00098E00E9456134C2F50E0FA013197E631F2
:1026E000F10580F5E25AFF4F0C94173788EE97E01A
:1026F00002C086ED97E00E9456132BC084EC97E051
:10270000FACF8AEB97E0F7CF89EA97E0F4CF8AE92E
:1027100097E0F1CF89E797E0EECF80E797E0EBCF46
:1027200085E697E0E8CF82E597E0E5CF84E497E09F
:10273000E2CF8EE297E0DFCF8AE197E0DCCF86E060
:1027400097E0D9CF84EF96E00E9456138C2F0E9419
:102750004A1381EF96E0CF910C945613CF938BEEF2
:1027600096E00E945613C0E06C2F84EC96E00E9425
:1027700087180E943B13C23021F089EE96E00E9438
:102780005613CF5FC33081F787EE96E00E94561351
:102790008091D0060E944A1383EE96E0CF910C946C
:1027A0005613FF920F931F93CF93DF938FED96E015
:1027B0000E945613809158060E944A1386EC96E0B8
:1027C0000E94561380915B060E944A1388EA96E0A5
:1027D0000E945613809159060E944A138FE896E092
:1027E0000E945613809159060E941F1388E896E0B4
:1027F0000E94561380915A060E944A1380E796E081
:102800000E94561380915A060E941F1389E696E093
:102810000E9456138091650682FB882780F90E94EA
:102820004A1388E496E00E9456138091650686FB61
:10283000882780F90E944A1388E296E00E94561386
:1028400080916506881F8827881F0E944A1388E0A8
:1028500096E00E94561380915C060E944A1382EF14
:1028600095E00E94561380915C060E941F138AEE29
:1028700095E00E94561360915D0670915E0680910E
:102880005F06909160060E94DD128AEC95E00E943E
:102890005613609161067091620680916306909173
:1028A00064060E94DD128FEA95E00E945613809123
:1028B000650681700E944A1382E995E00E945613D2
:1028C0008091650685FB882780F90E944A1387E777
:1028D00095E00E9456138091650683FB882780F956
:1028E0000E944A138CE595E00E945613809165067C
:1028F000829581700E944A1380E495E00E945613ED
:10290000809166060E944A1386E295E00E94561363
:10291000809166060E941F138EE195E00E94561377
:1029200060916706709168068091690690916A06C9
:102930000E94DD1281E095E00E94561360916D06C1
:1029400070916E0680916F06909170060E94DD1264
:1029500084EE94E00E945613809171060E944A13FF
:1029600085EC94E00E945613609173067091740692
:1029700080917506909176060E94DD128CEA94E0B3
:102980000E94561384E6F82EC0E008E216E0D0E07C
:102990008AEA94E00E9456138D2F8F0D0E944A13ED
:1029A00088EA94E00E945613C23079F0F801C330EF
:1029B000C1F0C13029F0608171818281938118C09A
:1029C000648575858685978513C020E030E041E6F3
:1029D00055E4F801608D718D828D938D0E9437389A
:1029E00007C084A195A1A6A1B7A1BC01CD019058B3
:1029F0000E94DD1285EA94E00E945613D13029F03E
:102A0000D23031F083EA94E005C081EA94E002C05C
:102A10008FE994E00E945613C23051F0C33059F050
:102A2000C13019F085E994E008C083E894E005C05E
:102A300082E794E002C082E694E00E9456138EE59D
:102A400094E00E945613DF5F0C5F1F4FD33009F0F4
:102A50009FCFFAE0FF0ECF5F8CE8F81296CFDF91A0
:102A6000CF911F910F91FF900895811104C088E0CC
:102A700098E00C9456130C9465132F923F924F924A
:102A80005F926F927F928F929F92AF92BF92CF92FE
:102A9000DF92EF92FF920F931F93CF93DF93CDB707
:102AA000DEB768970FB6F894DEBF0FBECDBFBB246C
:102AB000B39498E0792E20E2622E30E1A32E40E418
:102AC000542E52E0452E6CE0362E76E1272E1091E2
:102AD000B506112309F45BC0B092B20611FF07C01E
:102AE00084E094E00E94561389EF93E023C012FF24
:102AF00007C084E094E00E9456138EEE93E01AC063
:102B000013FF07C084E094E00E9456138BED93E01E
:102B100011C014FF07C084E094E00E94561380EDBA
:102B200093E008C015FF10C084E094E00E945613A3
:102B300084EC93E00E94561381EC93E00E945613BC
:102B400084EF91E00E948A0510FD08C08FB7F894C9
:102B50009091B5061092B5068FBF19C08FEB93E028
:102B60000E9456138DEA93E00E9456138CE493E082
:102B70000E9456139FB7F8948091B4068F7E80937D
:102B8000B4069FBF8091B40684FFFCCFDFCF1091C5
:102B9000B406112309F4E7C114FF04C081E0809357
:102BA000B106F2C110FF00C1E6EBF6E0DE011D96B2
:102BB000832D01900D928A95E1F78091B2068430C1
:102BC000E9F040F48130E9F080F0823009F589E3E2
:102BD00094E01CC0803179F018F4883049F018C0B6
:102BE000803291F0803421F013C088E594E00EC06B
:102BF00083E594E00BC08DE494E008C087E494E0A2
:102C000005C080E494E002C083E394E00E94561380
:102C100080915C06837039F0BE01635F7F4FCE0107
:102C200001960E94EA1880915C0680FD05C08091A3
:102C30005C0681FF6BC01FC08CE294E00E945613BB
:102C400069817A818B819C810E943B138AE294E0A6
:102C50000E9456136D817E818F8198850E943B135F
:102C60008AE294E00E94561369857A858B859C855B
:102C70000E943B13DCCF83E294E00E9456138CE069
:102C8000C82E86E0D82ECE0101967C0100E04701D7
:102C9000F60161917191819191916F01208531854A
:102CA000428553850E9438379B01AC01F701608152
:102CB0007181828193810E943737F701608371832C
:102CC00082839383023079F4209124063091250683
:102CD00040912606509127060E943737F7016083FE
:102CE000718382839383F4E0EF0EF11CF401608121
:102CF0007181828193810E943B13023021F081E235
:102D000094E00E9456130F5F033009F680915C0631
:102D100082FF0EC08BE194E00E9456138091AA04BA
:102D20009091A904891708F48E5E891B0E944A13AA
:102D300080915C0683FF0EC086E194E00E945613EA
:102D400090919F018091A001891708F48058891BF8
:102D50000E944A1380915C0684FF1AC080E194E0CF
:102D60000E94561393B196718091650686FF922555
:102D7000992349F091FB882780F992FD8260907138
:102D800019F0846001C080E043E062E00E94E0123C
:102D90008CE094E00E9456139FB7F8948091B4069B
:102DA0008E7F8093B4069FBF812F887609F444C03C
:102DB0008091B206882349F0982F9C77A9F188303A
:102DC00021F40E943E19B092B3068091B20681119F
:102DD00002C04092B30616FF09C0883011F4509229
:102DE000B2068091B30688608093B30613FF05C0D6
:102DF0008091B20685FFA092B20615FF15C08FEB39
:102E000093E00E9456138BE693E00E9456138CE4E5
:102E100093E00E9456138091B30681FD1460846094
:102E20008093B3066092B2069FB7F8948091B4067F
:102E300087798093B4069FBF11FF75C0812F887674
:102E400009F069C08091B206882339F0807509F4D1
:102E500062C08091B30681FF5EC08091B30682FF9D
:102E600020C08091F205882371F04091F3055091C4
:102E7000F4056091F5057091F6050E94172580EA2A
:102E80009FE00E948A058091F105882351F08230ED
:102E900011F4439A02C00E943C0688EE93E00E941F
:102EA0008A058091A9049091AA04981781F1F9E20A
:102EB000F89FC001112489539E4F892B41F18091C5
:102EC000B30683FD24C07092B2060E9460198091FF
:102ED000650682FF02C0289A01C028988091B20638
:102EE0008C70B9F08091A1018093B2018091A20110
:102EF0008093B10180915806880F8450819580930A
:102F0000B00180916F00826080936F0002C01092C8
:102F1000B2061092B3069FB7F8948091B4068D7FE5
:102F20008093B4069FBF12FF1EC08091B2068073CB
:102F300071F08091B30682FF04C00E9409250E94AF
:102F40003C068091B30682608093B30604C0109261
:102F5000B3061092B2069FB7F8948091B4068B7FA7
:102F60008093B4069FBF8091B2068C7711F00E94C7
:102F700060199091B2068091B306903219F481FDE8
:102F8000A092B2068111A3CD68960FB6F894DEBF69
:102F90000FBECDBFDF91CF911F910F91FF90EF90AA
:102FA000DF90CF90BF90AF909F908F907F906F9069
:102FB0005F904F903F902F9008954F925F926F9245
:102FC0007F928F929F92AF92BF92CF92DF92EF92B9
:102FD000FF920F931F93CF93DF9300D000D0CDB714
:102FE000DEB710916B068090B6069090B706A09061
:102FF000B806B090B906C090BA06D090BB06E09073
:10300000BC06F090BD06C701B601680D791D8A1D8A
:103010009B1D22E0422E512C612C712CA3019201A8
:103020000E94F83629833A834B835C83C501B4013F
:103030006C197D098E099F09A30192010E94F8363F
:103040008091BE069091BF06A091C006B091C106C6
:10305000113089F08092030190920401A092050141
:10306000B0920601C0920701D0920801E0920901D6
:10307000F0920A0114C0E980FA800B811C81E09271
:103080000301F092040100930501109306012093BF
:103090000701309308014093090150930A0180937E
:1030A0000B0190930C01A0930D01B0930E010F90B2
:1030B0000F900F900F90DF91CF911F910F91FF9084
:1030C000EF90DF90CF90BF90AF909F908F907F90C8
:1030D0006F905F904F900895CF93C0E08C2F0E9427
:1030E0001512811104C087E00E9465130AC0809107
:1030F0009905882331F00E9408120E949D060E94C3
:103100003515C13011F0C1E0E9CFCF9108950F938B
:103110001F93CF93DF93FC0180916B06813009F000
:1031200040C061111BC040815181628173818481E3
:103130009581A681B7818A019B01080F191F2A1F5B
:103140003B1FC901B8010E94E13820912806309147
:10315000290640912A0650912B061AC0613009F5C4
:1031600080819181A281B38104811581268137817B
:10317000BC01CD01601B710B820B930B0E94E138E7
:1031800020912C0630912D0640912E0650912F064D
:103190000E94373820E030E040E05FE30E948F3A41
:1031A00014C014E0619FE0011124EC0FFD1F608149
:1031B0007181828193810E94E138C85DD94F288155
:1031C00039814A815B810E943738DF91CF911F910D
:1031D0000F910895EF92FF920F931F93CF937B016E
:1031E0008C01C0E06C2FC7010E948718F801619321
:1031F0007193819391938F01CF5FC33099F7CF91F2
:103200001F910F91FF90EF9008951F920F920FB6AC
:103210000F9211242F933F934F935F936F937F935C
:103220008F939F93AF93BF93EF93FF9386B1809556
:10323000877099F080FF03C00E943E060EC0982F51
:10324000947021F08091B406826005C081FF05C0B2
:103250008091B40688608093B406FF91EF91BF918E
:10326000AF919F918F917F916F915F914F913F911E
:103270002F910F900FBE0F901F901895CF93DF9353
:10328000C0916C05D0916D052097B9F081E08093D5
:103290006F056091850570918605809187059091F5
:1032A00088059B01AC010E948F3A698B7A8B8B8BCE
:1032B0009C8B10926D0510926C05DF91CF91089553
:1032C0002F923F924F925F926F927F928F929F9236
:1032D000AF92BF92CF92DF92EF92FF920F931F9324
:1032E000CF93DF93CDB7DEB7CE54D1090FB6F894A4
:1032F000DEBF0FBECDBF8091B206807725968FAF1F
:103300002597882389F020E030E0A90160918505A8
:103310007091860580918705909188050E942D38CF
:10332000882311F40C943222209185052B8B309147
:1033300086053C8B409187054D8B509188055E8BAF
:10334000809195058B83909196059D83A09197051B
:10335000AE83B0919805BC830091810510918205E0
:103360005091830540918405809174059091750575
:10337000A0917605B09177058FA398A7A9A7BAA7C2
:10338000909170059FAFA09171052196AFAF2197E5
:10339000B09172052296BFAF2297E09173052396F4
:1033A000EFAF239780917C0590917D05A0917E05DC
:1033B000B0917F058FAB98AFA9AFBAAF90911405CC
:1033C00024969FAF2497A091EF04ADA7B091AA04D3
:1033D0002796BFAF2797E091A904E8A3F091C60113
:1033E0002696FFAF269720916C0530916D053A8B9C
:1033F000298B80911505909116059AA389A3809138
:10340000780590917905A0917A05B0917B058BAFF5
:103410009CAFADAFBEAF90918D059F8BA0918E05F7
:10342000A88FB0918F05B98FE0919005EA8F309009
:10343000910520909205F0919305F98320919405D0
:103440002A83309189053B8F80918A058C8F9091DA
:103450008B059D8FA0918C05AE8F8091EE049DA56C
:10346000891709F466C7E989FA89EF2B09F089C23F
:103470002796FFAD279728A1F21781F0A22EB12C35
:1034800039E23A9DC0013B9D900D1124DC01A95306
:10349000BE4FBA8BA98BAB2B09F051C0C801A52F29
:1034A000B42F8093810590938205A0938305B093F8
:1034B00084058F89988DA98DBA8D80938D05909301
:1034C0008E05A0938F05B09390058B899C89AD895B
:1034D000BE898093850590938605A0938705B09358
:1034E00088058B8D9C8DAD8DBE8D809389059093C5
:1034F0008A05A0938B05B0938C058B819D81AE814D
:10350000BC818093950590939605A0939705B09301
:103510009805832D922DA981BA818093910590936E
:103520009205A0939305B09394052496BFAD24977C
:10353000B093140510926D0510926C054CC78091E4
:103540006F05882319F010926F05BFC080916E053A
:103550008F5F853019F080936E0502C010926E0562
:1035600080916E0551E1589FC0011124DC01A95ED4
:10357000BA4FBAA3A9A3B9E2BA9D9001BB9D300D81
:103580001124F901E953FE4F7F018081A9A1BAA15D
:103590008C9381819281A381B48123E0880F991F4C
:1035A000AA1FBB1F2A95D1F7E9A1FAA181839283B3
:1035B000A383B483F70185819681A781B08533E029
:1035C000880F991FAA1FBB1F3A95D1F7E9A1FAA14D
:1035D00085839683A783B087F70181859285A3852C
:1035E000B48543E0880F991FAA1FBB1F4A95D1F7E6
:1035F000E9A1FAA181879287A387B487D7011D9695
:103600006D917D918D919C9150978B019C0153E020
:10361000000F111F221F331F5A95D1F705871687F8
:103620002787308B0E94DF386FAF21967FAF2197BD
:1036300022968FAF229723969FAF2397D701959617
:103640002D913D914D915C9198970E9437386FA3D1
:1036500078A789A79AA79B01AC0160E070E080EA97
:103660009FE30E9437386BAF7CAF8DAF9EAF25963E
:10367000BFAD2597BB23C1F02F89388D498D5A8D59
:103680006F89788D898D9A8D0E948F3AF701618BB1
:10369000728B838B948BFF89FB8B288D2C8B398DC0
:1036A0003D8B4A8D4E8B0DC0D70151966D917D910A
:1036B0008D919C9154970E942E3B6B8B7C8B8D8BB4
:1036C0009E8B1FAA18AE19AE1AAEB9E2BA9D900130
:1036D000BB9D300D1124F901E953FE4F4F01C1A0EC
:1036E000D2A0E3A0F4A0A701960160E070E080E022
:1036F0009FE30E94373869877A878B879C87259656
:10370000FFAD2597FF23E9F122E020938005D40146
:1037100095964D905D906D907C90989751968D9078
:103720009D90AD90BC905497A50194010E948F3A52
:103730009B01AC01C301B2010E9437378B0189871D
:103740009D8720E030E0A9010E942D3887FF1EC12F
:10375000A7019601C701B6010E943837A301920163
:103760000E948F3A9B01AC01C501B4010E9437371A
:103770000E942E3B6F8B788F898F9A8F3F8228868D
:1037800018C110928005F401F5A1FF83D40196962B
:10379000BC91B887F40107A110A5E8A1EF5FE23161
:1037A00009F4E0E02796FFAD2797EF1789F029E2AB
:1037B0002E9FF0011124E953FE4F6189728983899C
:1037C00094890E942E3B6F8B788F898F9A8F04C0CB
:1037D0001F8A188E198E1A8E2F89388D498D5A8D11
:1037E0006F89788D898D9A8D0E948F3A2B013C01CB
:1037F00049E24A9D90014B9D300D1124C901895326
:103800009E4F5C01DC0151962D913D914D915C9153
:1038100054972D873E874F87588BA30192016D8562
:103820007E858F8598890E9437379B01AC01698519
:103830007A858B859C850E948F3A9B01AC016F81B4
:103840007885C8010E94383720E030E040E05FE32F
:103850000E948F3A362E272E89839A8320E030E00B
:10386000A9010E944F3A18160CF097C02F81388595
:10387000A801632D722D89819A810E942D3887FFBE
:1038800072C0F501858C968CA78CB0A0A301920123
:10389000C501B4010E9437379B01AC0169857A8567
:1038A0008B859C850E948F3A6B837D838E839C835E
:1038B000232D322D49815A810E942D3887FF34C033
:1038C000C501B4010E942E3B6B8F7C8F8D8F9E8F24
:1038D000A50194016D857E858F8598890E942D387C
:1038E000811106C0F1E0F093800509831A8361C05D
:1038F0002D853E854F855889C501B4010E94373713
:103900009B01AC0169857A858B859C850E948F3AE5
:103910009B01AC016F817885C8010E9437376F83A6
:10392000788789839A8345C0A7019601C701B601AC
:103930000E943837232D322D49815A810E948F3AB7
:10394000A30192010E9438370E942E3B6B8F7C8F1F
:103950008D8F9E8F3F8228863B822D8229812E83E8
:103960003A813C8326C042E04093800509831A8354
:103970005B895B8F8C898C8F9D899D8FAE89AE8F83
:1039800018C03F82288659874D8717C03F822886F6
:103990001F8A188E198E1A8E10C0BF89BB8FE88DB2
:1039A000EC8FF98DFD8F2A8D2E8F1F82188619823C
:1039B0001A8200E010E019861D8624965FAD2497D8
:1039C000452F50E05CA74BA786E0849FF001859FC0
:1039D000F00D1124E051FB4F80916E058283A9897F
:1039E000BA899596BC91BAABE989FA89F6A1FBAB85
:1039F000A989BA899796BC912896BFAF2897E9897B
:103A0000FA89F0A52996FFAF29972BAD3CAD4DADB6
:103A10005EAD6AA97BA98B2F9F2F0E9437376EA7B7
:103A20007FA788AB99AB20E030E0A9010E942D3838
:103A300087FF04C01EA61FA618AA19AA20918005F8
:103A40002F8F2AA83BA92F963FAF2F9728964FADCF
:103A500028972E964FAF2E9729963FAC29978EE345
:103A6000C82E83ECD82E8EE2E82E89E3F82E412C66
:103A7000512C3201CBA2DCA2EDA2FEA29F8D992394
:103A800021F0913009F496C0D6C0A989BA899196DF
:103A90002D913D914D915C919497C701B6010E9483
:103AA0008F3A4B015C0120E030E040E05FE30E9490
:103AB0008F3A9B01AC016B897C898D899E890E941C
:103AC00038379B01AC01C701B6010E948F3A9B01B8
:103AD000AC01622D2F967FAD2F972E968FAD2E972E
:103AE000932D0E943737262E2F967FAF2F972E9635
:103AF0008FAF2E97392E2F81388549815A810E94A8
:103B00002D3887FF4AC02F81388549815A816AA99B
:103B10007BA928968FAD289729969FAD29970E945B
:103B200037379B01AC010E9438376B017C012B8D2C
:103B30003C8D4D8D5E8D6B897C898D899E890E941F
:103B400038379B01AC01C701B6010E9437386B01C1
:103B50007C012B813D814E815C816F8178858981DB
:103B60009A810E942D38811103C0B2E0BF8F02C03C
:103B7000E1E0EF8FFB8DFB8B2C8D2C8B3D8D3D8BF6
:103B80004E8D4E8B2F8058852F965FAF2F97898152
:103B90002E968FAF2E973A80F0C0A50194016B89C5
:103BA0007C898D899E890E9438376B8B7C8B8D8BAD
:103BB0009E8BE3C0A70196016B8D7C8D8D8D9E8DB4
:103BC0000E948F3A9B01AC01622D2F967FAD2F97FB
:103BD0002E968FAD2E97932D0E9437374B015C01A7
:103BE0002B813D814E815C810E942D3887FFBDC0B5
:103BF0002B813D814E815C81622D2F967FAD2F9769
:103C00002E968FAD2E97932D0E9437372B8D3C8D9E
:103C10004D8D5E8D0E9437386B017C012B809D811C
:103C20002F969FAF2F97AE812E96AFAF2E973C80E9
:103C3000B2E0BF8FA2C0E989FA8921A132A143A1D4
:103C400054A1C701B6010E948F3A4B015C019B0150
:103C5000AC016B897C898D899E890E944F3A181628
:103C60000CF054C020E030E040E05FE3C501B40157
:103C70000E948F3A9B01AC016B897C898D899E895A
:103C80000E9437379B01AC01C701B6010E948F3AF1
:103C90009B01AC01622D2F967FAD2F972E968FAD95
:103CA0002E97932D0E9437372A966FAF2A972B961F
:103CB0007FAF2B972C968FAF2C972D969FAF2D977C
:103CC000980149855D850E944F3A1816FCF4A501BC
:103CD00094016B897C898D899E890E9437376B8B13
:103CE0007C8B8D8B9E8B2A962FAC2A972B96FFADC3
:103CF0002B972F96FFAF2F972C962FAD2C972E96A4
:103D00002FAF2E972D963FAC2D9737C09801498540
:103D10005D85622D2F967FAD2F972E968FAD2E97B6
:103D2000932D0E9437379B01AC010E9438376B01FD
:103D30007C012F89388D498D5A8D6B897C898D89BD
:103D40009E890E9438379B01AC01C701B6010E94D1
:103D500037386B017C01202E2F961FAF2F973985A6
:103D60002E963FAF2E973D8408C0282C2F969FAEED
:103D70002F972E96AFAE2E973B2CA7019601C3012D
:103D8000B2010E9438372B013C012BA13CA14DA16F
:103D90005EA10E942D3887FF07C0A30192016BA18D
:103DA0007CA18DA19EA163C02EA53FA548A959A9BC
:103DB000622D2F967FAD2F972E968FAD2E97932D38
:103DC0000E944F3A18160CF442C04F8D4093800564
:103DD000222D2F963FAD2F972E964FAD2E97532D18
:103DE0006FA178A589A59AA50E948F3A6F8F7BA3B2
:103DF0008EA79AAB0E9416386B017C016FAD21969D
:103E00007FAD219722968FAD229723969FAD239762
:103E10000E9416384B015C01A70196010E943737BA
:103E20000E94B0386BAB7CAB8DAB9EABA6E08BA594
:103E30009CA5A89FF001A99FF00D1124E051FB4F14
:103E40002BA93CA931832083232B49F1B5C02EE354
:103E500033EC4EE259E36BA17CA18DA19EA10E949F
:103E600038376BA37CA38DA39EA3A30192010E946C
:103E700037376B017C01980149855D85622D2F964E
:103E80007FAD2F972E968FAD2E97932D0E944F3A90
:103E900018160CF4F3CD5F8D5093800599CF2596BD
:103EA0008FAD2597882309F487C0C801A985BD85F2
:103EB0008093810590938205A0938305B093840538
:103EC0008F89988DA98DBA8D80938D0590938E05DD
:103ED000A0938F05B09390058B8D9C8DAD8DBE8D7D
:103EE0008093890590938A05A0938B05B0938C05E8
:103EF0008B819D81AE81BC818093950590939605C1
:103F0000A0939705B09398058F819885A981BA8170
:103F10008093910590939205A0939305B093940597
:103F200024969FAD249790931405A989BA89B093DC
:103F30006D05A0936C052BAD3CAD4DAD5EAD2093F2
:103F400078053093790540937A0550937B0538A125
:103F50003093A90449A15AA1509316054093150521
:103F60008FA198A5A9A5BAA580937405909375050E
:103F7000A0937605B09377059DA59093EF041092DA
:103F8000850510928605109287051092880510927B
:103F90007C0510927D0510927E0510927F05C092DF
:103FA0007005D0927105E0927205F09273052FA111
:103FB00038A549A55AA56FC12FA938AD49AD5AAD4D
:103FC000C301B2010E9438372B013C012F8D3BA168
:103FD0004EA55AA9C501B4010E9437379B01AC0117
:103FE000C301B2010E9437384B015C012F8D3BA108
:103FF0004EA55AA9C701B6010E943737A501940101
:104000000E948F3A6FAB78AF89AF9AAF20EC31EE58
:1040100044E65EE4C501B4010E948F3A0E9416385E
:104020000E94B038603DB7E07B078105910560F4E0
:1040300046E02BA53CA5429FF001439FF00D1124C3
:10404000E051FB4F158253C0603A5FE07507810570
:10405000910560F426E0ABA5BCA52A9FF0012B9F3B
:10406000F00D1124E051FB4F31E011C060344FE1FD
:1040700074078105910568F426E0ABA5BCA52A9FCD
:10408000F0012B9FF00D1124E051FB4F32E03583FE
:104090000CC0A6E04BA55CA5A49FF001A59FF00D68
:1040A0001124E051FB4FB3E0B58346E02BA53CA5BE
:1040B000429FF001439FF00D1124E051FB4F2581F9
:1040C000022E04C096958795779567950A94D2F746
:1040D000ABA9BCA902C0AA0FBB1F2A95E2F7B18306
:1040E000A08361157105B1E08B07910568F446E086
:1040F0002BA53CA5429FF001439FF00D1124E051F8
:10410000FB4F7483638304C08FEF9FEF948383839B
:10411000BDA4B39496E0B91201C0B12C98014985B1
:104120005D85622D2F967FAD2F972E968FAD2E97A2
:10413000932D0E944F3A1816ECF4822D2F969FADC6
:104140002F972E96AFAD2E97B32DE989FA8985A3C7
:1041500096A3A7A3B0A7FF8DFFAF2BA121962FAFEA
:1041600021973EA522963FAF22974AA923964FAFAB
:104170002397D5C020E030E0A901622D2F967FADB6
:104180002F972E968FAD2E97932D0E944F3A18168B
:104190000CF0AEC0C801A985BD85809381059093C0
:1041A0008205A0938305B09384058F89988DA98D8E
:1041B000BA8D80938D0590938E05A0938F05B09353
:1041C00090058B8D9C8DAD8DBE8D809389059093D0
:1041D0008A05A0938B05B0938C058B819D81AE8160
:1041E000BC818093950590939605A0939705B09315
:1041F00098058F819885A981BA81809391059093C4
:104200009205A0939305B09394055DA55093140572
:1042100089899A8990936D0580936C052BAD3CAD8F
:104220004DAD5EAD209378053093790540937A05C6
:1042300050937B0538A13093A90449A15AA150930A
:104240001605409315058FA198A5A9A5BAA5809339
:10425000740590937505A0937605B0937705B09299
:10426000EF04109285051092860510928705109232
:10427000880510927C0510927D0510927E051092A3
:104280007F05C0927005D0927105E0927205F092A0
:1042900073059C01AD01C701B6010E943738A98999
:1042A000BA8995966D937D938D939C9398970E9470
:1042B0003E198091A9048093C601C25BDF4F0FB6FF
:1042C000F894DEBF0FBECDBFDF91CF911F910F914C
:1042D000FF90EF90DF90CF90BF90AF909F908F9026
:1042E0007F906F905F904F903F902F900C943F0481
:1042F0002796BFAD2797E8A1BE1779F08E2F8F5F65
:10430000823109F480E0F8A126962FAD2697F213AA
:1043100003C026968FAF269788A31A8A198A5985D3
:104320004D853F8028843DA524963FAF2497BDA6A8
:1043300094C8C801A52FB42F80938105909382055E
:10434000A0938305B09384058F89988DA98DBA8D2C
:1043500080938D0590938E05A0938F05B093900563
:104360008B899C89AD89BE8980938505909386054C
:10437000A0938705B09388058B8D9C8DAD8DBE8DE8
:104380008093890590938A05A0938B05B0938C0543
:104390008B819D81AE81BC8180939505909396051C
:1043A000A0939705B0939805832D922DA981BA818A
:1043B0008093910590939205A0939305B0939405F3
:1043C0002496AFAD2497A0931405E989FA89F09358
:1043D0006D05E0936C052BAD3CAD4DAD5EAD20930E
:1043E00078053093790540937A0550937B0538A181
:1043F0003093A90449A15AA150931605409315057D
:104400008FAD21969FAD21972296AFAD229723962F
:10441000BFAD23978093700590937105A0937205AB
:10442000B09373058FA198A5A9A5BAA5809374052B
:1044300090937505A0937605B09377052FA938ADB5
:1044400049AD5AAD20937C0530937D0540937E05A0
:1044500050937F053DA53093EF0426964FAD2697E8
:104460004093C601C25BDF4F0FB6F894DEBF0FBEAC
:10447000CDBFDF91CF911F910F91FF90EF90DF9013
:10448000CF90BF90AF909F908F907F906F905F90F4
:104490004F903F902F90089580915906682F90E09B
:1044A00020915A06422F80FD94E0822F817020FDDA
:1044B00080E261FD986041FD806462FD906142FD93
:1044C00080689093A2018093A10108951F920F929A
:1044D0000FB60F9211248F939F938BB19091A201ED
:1044E0009C71837E892B8BB915BC9F918F910F9006
:1044F0000FBE0F901F90189580916F008D7F809355
:104500006F0080918100887F81608093810010928C
:10451000ED0480915B068F3F21F49091B5069923BD
:1045200049F09091B206943029F090E00E948A05FB
:1045300081E001C080E09091650692FF02C091E0A9
:104540008927882311F0289A0895289808950E94B1
:104550007C228BE2EEE6F5E0DF011D928A95E9F719
:1045600083E2E3EAF1E0DF011D928A95E9F7109218
:104570006D0510926C051092EE041092140581E006
:104580008093EF041092ED040E944C228BB1837E45
:104590009091A201892B8BB98BB18F719091A10160
:1045A000892B8BB908951F920F920FB60F92112489
:1045B0002F933F934F935F936F937F938F939F932B
:1045C000AF93BF93EF93FF938091ED04811110C2DD
:1045D0008BB19091B201907E8F71892B8BB98BB189
:1045E000837E9091B101892B8BB98091B00186BDFA
:1045F00082E085BD81E08093ED0478948091C401D0
:104600009091C501892B09F0ADC08091EE04909185
:104610001405981709F49BC0E091EE042E2F30E0AA
:1046200086E0E89FF0011124E051FB4FF093C501B3
:10463000E093C401838194819093890080938800E2
:10464000808191819093C0018093BF01E28180912C
:10465000C1018E1761F1E093C10181E1E89FF00192
:104660001124E95EFA4FF093C301E093C2018585FE
:104670009685A785B089B695A795979587958093D8
:10468000AB019093AC01A093AD01B093AE018093C8
:10469000A7019093A801A093A901B093AA018093C8
:1046A000A3019093A401A093A501B093A601E0916A
:1046B000C201F091C3019091A1018081892780936B
:1046C000B20186E0829FD001839FB00D1124A051DA
:1046D000BB4F15962C9181819281A381B481022ECA
:1046E00004C0B695A795979587950A94D2F78093BD
:1046F000B3019093B401A093B501B093B601858145
:104700009681A781B085022E04C0B695A79597958E
:1047100087950A94D2F78093B7019093B801A0933C
:10472000B901B093BA0181859285A385B48504C08F
:10473000B695A795979587952A95D2F78093BB0153
:104740009093BC01A093BD01B093BE010BC00E9429
:104750007C229FB7F8948091B40684608093B4065D
:104760009FBF46C18091C3068130B1F486B180728B
:1047700090917706891781F01092C3068CE0E6EBE2
:10478000F6E0A4ECB6E001900D928A95E1F78091F5
:10479000B40680648093B4061092B1014091B301D5
:1047A0005091B4016091B5017091B6018091A3015F
:1047B0009091A401A091A501B091A601840F951F2D
:1047C000A61FB71F8093A3019093A401A093A501F6
:1047D000B093A601E091C201F091C30145855685D1
:1047E00067857089481759076A077B0768F524E0D1
:1047F0002093B1014585568567857089841B950B8B
:10480000A60BB70B8093A3019093A401A093A501DD
:10481000B093A60120818091B6069091B706A09131
:10482000B806B091B90625FF04C00197A109B109E6
:1048300003C00196A11DB11D8093B6069093B706E3
:10484000A093B806B093B9064091B7015091B80152
:104850006091B9017091BA018091A7019091A8016E
:10486000A091A901B091AA01840F951FA61FB71F9F
:104870008093A7019093A801A093A901B093AA01E6
:104880004585568567857089481759076A077B07EC
:1048900078F52091B10128602093B10145855685B6
:1048A00067857089841B950BA60BB70B8093A701B6
:1048B0009093A801A093A901B093AA0120818091AF
:1048C000BA069091BB06A091BC06B091BD0626FF2A
:1048D00004C00197A109B10903C00196A11DB11D32
:1048E0008093BA069093BB06A093BC06B093BD0616
:1048F0004091BB015091BC016091BD017091BE011E
:104900008091AB019091AC01A091AD01B091AE014D
:10491000840F951FA61FB71F8093AB019093AC0126
:10492000A093AD01B093AE0145855685678570892A
:10493000481759076A077B0778F52091B101206174
:104940002093B1014585568567857089841B950B39
:10495000A60BB70B8093AB019093AC01A093AD0174
:10496000B093AE0120818091BE069091BF06A091C8
:10497000C006B091C10627FF04C00197A109B10983
:1049800003C00196A11DB11D8093BE069093BF0682
:10499000A093C006B093C1068091B206843039F46A
:1049A0009091C2068091B10189238093B1018091D9
:1049B000BF019091C00101979093C0018093BF0106
:1049C000892B69F41092C5011092C4018091EE0404
:1049D0008F5F8093EE04863011F41092EE04909174
:1049E000A2018091B10189278093B1011092ED0459
:1049F000FF91EF91BF91AF919F918F917F916F91B7
:104A00005F914F913F912F910F900FBE0F901F908C
:104A1000189580916C06813021F48FE08093B3006B
:104A200008958091B0008F778093B0000895CF9261
:104A3000DF92EF92FF926A017B01811106C0FF9025
:104A4000EF90DF90CF900C940925813011F42D98D0
:104A500001C02D9A83E88093B0008091B100887FD7
:104A600082608093B10020E030E0A901C701B60167
:104A70000E942D3818161CF720E030E0A901C7016C
:104A8000B6010E942D3887FD11C020E030E044EBD4
:104A900052E4C701B6010E944F3A181654F4C12CD3
:104AA000D12C84EBE82E82E4F82E03C0C12CD12C4B
:104AB000760125E535E545E350E4C701B6010E94DE
:104AC0008F3A20E030E040E05FE30E9438370E94F8
:104AD0001C390E94B0386093B300FF90EF90DF90D4
:104AE000CF90089569E080E090E00E94DB054FE4FC
:104AF00050E068E276E081E090E00C94FD052DE066
:104B0000829FC00111244CE050E09E5F0C94FD0593
:104B10001F93CF93DF93182FEB018DE0189FB00107
:104B200011247E5F4CE050E0CE010E949505892B58
:104B300059F48CE0FE0111928A95E9F7BE01812FAC
:104B40000E947F2580E001C081E0DF91CF911F911D
:104B50000895EF92FF920F931F93CF93DF93CDB7FA
:104B6000DEB72C970FB6F894DEBF0FBECDBF182F5F
:104B700080FFCDC08AE08093580689E180935B0670
:104B80001092590610925A0683E080935C068AE0E0
:104B900097EDA3E2BCE380935D0690935E06A0933D
:104BA0005F06B09360068FE692E1A3E0BBE38093DB
:104BB000610690936206A0936306B0936406109218
:104BC000660680E090E0A8ECB1E4809367069093DD
:104BD0006806A0936906B0936A0610926B0610925D
:104BE0006C0680E090E0AAEFB3E480936D069093AA
:104BF0006E06A0936F06B09370068AEF90E09093D4
:104C000072068093710680E090E0A0E8BFE3809395
:104C1000730690937406A0937506B093760610926F
:104C2000650680E090E0A0EAB2E4809328069093C5
:104C30002906A0932A06B0932B0680932C06909306
:104C40002D06A0932E06B0932F0680E090E0A8ECEE
:104C5000B3E48093300690933106A0933206B0936C
:104C6000330680E090E4ACE9B5E480933406909399
:104C70003506A0933606B093370680933806909396
:104C80003906A0933A06B0933B0680933C06909376
:104C90003D06A0933E06B0933F0680E098ECAFE25D
:104CA000B9E48093400690934106A0934206B093E6
:104CB00043068093440690934506A0934606B0931E
:104CC00047068093480690934906A0934A06B093FE
:104CD0004B0680E090E4ACE9B5EC80934C069093F1
:104CE0004D06A0934E06B0934F06809350069093C6
:104CF0005106A0935206B0935306809354069093A6
:104D00005506A0935606B09357060E94722511FFD0
:104D100010C0CE0101967C018CE0F70111928A95BA
:104D2000E9F700E0B701802F0E947F250F5F083070
:104D3000C9F712FF0AC060E080E093E00E94DB0543
:104D400060E081E593E00E94DB0513FF05C060E0B1
:104D50008EEA93E00E94DB052C960FB6F894DEBF36
:104D60000FBECDBFDF91CF911F910F91FF90EF90BC
:104D700008951F920F920FB60F9211242F933F9315
:104D80004F935F936F937F938F939F93AF93BF9353
:104D9000EF93FF938091C6008F33A9F050F48831D0
:104DA00009F1813211F59FB7F8948091B4068860BB
:104DB00015C0803471F08E37C1F49FB7F89480919C
:104DC000B40682600BC09FB7F8948091B4068160EE
:104DD00005C09FB7F8948091B40680628093B406B2
:104DE0009FBF14C00E943E0611C0E091A00191E057
:104DF0009E0F903809F490E020919F01921731F0B6
:104E0000F0E0E15EFE4F80839093A001FF91EF916F
:104E1000BF91AF919F918F917F916F915F914F91D2
:104E20003F912F910F900FBE0F901F9018951F92DA
:104E30000F920FB60F9211248F939F93EF93FF93CE
:104E40008091EC04E82FF0E0E455FB4F90819093C3
:104E5000C6008F5F803409F480E08093EC04909169
:104E6000AB04891305C08091C1008F7D8093C10080
:104E7000FF91EF919F918F910F900FBE0F901F9018
:104E80001895E091AB0491E09E0F903431F490E0DE
:104E900004C02091B40624FD0FC02091EC049217A9
:104EA000C1F3F0E0E455FB4F80839093AB04809115
:104EB000C10080628093C10008958F929F92AF924B
:104EC000BF92CF92DF92EF92FF920F931F93CF93F7
:104ED000DF937C016B01DC01EC91F0E0E756FA4FC7
:104EE0009081EF019D3221F42296918101E007C06B
:104EF0009B3211F0219602C02296918100E0912C04
:104F0000F0E010E020E030E0A9015E01E0EDE90F03
:104F1000EA30D0F4FF5FF93098F491101150A5E019
:104F2000B0E00E941D37DC01CB01880F991FAA1F3A
:104F3000BB1F9C01AD012E0F311D411D511D0AC02B
:104F4000911008C01F5F06C0EE3F41F4911006C0EB
:104F5000992493942196D5019C91D7CFFF2309F4EE
:104F60004FC0CA01B9010E94DF384B015C0120E04B
:104F700030E0A9010E942D38882349F11F3F64F4D5
:104F80002AE037ED43E25CE3C501B4010E948F3AA9
:104F90004B015C011E5FF2CF1F3F59F42DEC3CEC3E
:104FA0004CEC5DE3C501B4010E948F3A4B015C01FA
:104FB0000EC0112361F020E030E040E251E4C50171
:104FC000B4010E948F3A4B015C011150F2CF0023D3
:104FD00051F0B7FAB094B7F8B094F601808291829C
:104FE000A282B38206C0D6018D929D92AD92BC92F0
:104FF0001397C959D540C150F701C08381E001C062
:1050000080E0DF91CF911F910F91FF90EF90DF90A3
:10501000CF90BF90AF909F908F9008952F923F9226
:105020004F925F926F927F928F929F92AF92BF92B8
:10503000CF92DF92EF92FF920F931F93CF93DF9364
:10504000CDB7DEB7C954D1090FB6F894DEBF0FBE95
:10505000CDBF9E8F8D8F49A35AA36BA37CA32896A7
:105060002FAF28978091650685FF28C00D8D1E8D76
:105070009CE4E92E96E0F92E68012CE0C20ED11CCA
:10508000D8018D909D90AD90BD908D0120E030E0D5
:10509000A901C501B4010E944F3A18161CF1F7018D
:1050A00021913191419151917F01C501B4010E943B
:1050B0002D3887FD17C00C151D0511F78091B2061C
:1050C000823009F4BEC40E943D158091B106811161
:1050D000B8C49091A90480910201981326C00E943F
:1050E0002313F1CF8091B206883091F49FB7F894E2
:1050F0008091B40688608093B4069FBF0E943D15DE
:105100008091B1068111DACF8091B2068111F6CF7C
:105110000E943E069FB7F8948091B5068560809303
:10512000B5069FBF0E943D15C9CFF090AA042F2C51
:10513000312C99E2F99E8001112409531E4FD801A8
:105140001D961D921D921D921C925097F80115A25A
:1051500016A217A210A6108289E996E7A6E9BEE773
:1051600081A392A3A3A3B4A380916B062091030112
:105170003091040140910501509106012FAB38AFE9
:1051800049AF5AAF8090070190900801A0900901A3
:10519000B0900A01813009F070C02091280630914A
:1051A000290640912A0650912B06AD8DBE8D6D913A
:1051B0007D918D919C910E948F3A0E945C3A2B01C7
:1051C0003C016D877E878F87988B20912C063091CC
:1051D0002D0640912E0650912F06ED8DFE8D648197
:1051E0007581868197810E948F3A0E945C3AAB015B
:1051F000BC01498B5A8B6B8B7C8B8FA998ADA9AD69
:10520000BAAD481A590A6A0A7B0ADB01CA01881931
:105210009909AA09BB09840D951DA61DB71DB7FFE5
:1052200007C0B095A095909581959F4FAF4FBF4F08
:10523000F80181839283A383B48389E2829DF00184
:10524000839DF00D1124E953FE4FD501C401841B49
:10525000950BA60BB70B480E591E6A1E7B1E77FED8
:1052600008C07094609450944094411C511C611C7F
:10527000711C458256826782708600916B06209170
:105280003006309131064091320650913306239614
:105290002CAF3DAF4EAF5FAF239780910B01909144
:1052A0000C01A0910D01B0910E0127968CAF9DAF1E
:1052B000AEAFBFAF2797DE011196BEA3ADA3E8E264
:1052C000F6E0FEA7EDA79E01235F3F4F38A72FA36F
:1052D00043E051E05CAB4BABCD8CDE8CDEAACDAABB
:1052E00029E2F29EC0011124AC0149535E4F58AB34
:1052F0004FA783E091E09CA78BA7FC8FEB8FCDA0FD
:10530000DEA0DEAECDAE10E029E2229DC001239DDD
:10531000900D11249C0129533E4F38A32F8F235FFA
:105320003F4F3AAB29AB4F8D58A1475F5F4F2A964D
:105330005FAF4EAF2A978F8D98A185969CAF8BAFAC
:10534000013009F09FC0123099F5AD8DBE8D1896D1
:105350002D913D914D915C911B9723966CAD7DAD48
:105360008EAD9FAD23970E948F3A0E945C3A6D8B61
:105370007E8B8F8B988FDC01CB012796CCACDDAC7C
:10538000EEACFFAC27978C199D09AE09BF09B7FF9A
:1053900007C0B095A095909581959F4FAF4FBF4F97
:1053A0002A96EEADFFAD2A9780839183A283B383C3
:1053B000A9A9BAA94D915D916D917C91EFA5F8A92C
:1053C00081819281A381B48184179507A607B707CD
:1053D00010F4DB01CA01E9A9FAA980839183A283B1
:1053E000B383111117C08D859E85AF85B889AC0137
:1053F000BD01CFA8D8ACE9ACFAAC4C195D096E0977
:105400007F0989899A89AB89BC8988199909AA0970
:10541000BB091CC0113019F58D859E85AF85B889F3
:10542000AC01BD01CFA8D8ACE9ACFAAC4C195D0910
:105430006E097F0989899A89AB89BC8975016401E4
:10544000C81AD90AEA0AFB0AD701C6016A017B0118
:10545000C80ED91EEA1EFB1EC701B60157C0EFA138
:10546000F8A580819181A281B381EBA5FCA5C080C4
:10547000D180E280F380BC01CD016C197D098E09D9
:105480009F0944C0EB8DFC8D208131814281538185
:10549000ADA9BEA96D917D918D919C910E948F3A8D
:1054A0000E945C3AEFA1F8A56083718382839383A5
:1054B000ABA5BCA5CD90DD90ED90FC906C197D095D
:1054C0008E099F096B017C0197FF07C0CC24DD2466
:1054D0007601C61AD70AE80AF90AEFA5F8A9C18227
:1054E000D282E382F482A9A9BAA94D905D906D9011
:1054F0007C90C414D504E604F70410F4730162012F
:10550000E9A9FAA9C082D182E282F3820E94E1383D
:10551000AB8DBC8D2D913D914D915C910E943738A2
:105520006B017C01EDADFEAD61937193819391931D
:10553000FEAFEDAF20E030E0A9010E942D3887FFDB
:105540000EC0112321F0113021F090E803C090E249
:1055500001C090E4AF8DB8A18C91892B8C93A701E9
:105560009601C701B6010E948F3AEBADFCAD2081D8
:105570003181428153810E943837ABADBCAD6D9310
:105580007D938D939C9313971F5FEB8DFC8D3496C9
:10559000FC8FEB8F2FA138A52C5F3F4F38A72FA38F
:1055A0004BA55CA54C5F5F4F5CA74BA7ADA9BEA9FF
:1055B0001496BEABADABEFA5F8A93496F8ABEFA748
:1055C000133009F0BDCE0E942E3B6B017C01ABADC8
:1055D000BCAD6D937D938D939C931397EF8DF8A144
:1055E00085859685A785B089892B8A2B8B2B09F415
:1055F00028C220E030E0A90169A17AA18BA19CA179
:105600000E942D3887FD24C02896FFAD2897FF23E0
:1056100061F0A701960169A17AA18BA19CA10E94CA
:105620008F3A69A37AA38BA39CA320E030E040E8E3
:105630005FE369A17AA18BA19CA10E942D3887FF0D
:105640000FC019A21AA220E82BA33FE33CA308C075
:1056500049E949A356E75AA386E98BA39EE79CA391
:10566000A701960160E070E080E89FE30E94373870
:105670006FA378A789A79AA7DE011D96BA8FA98F75
:10568000C12CD12C760129E2229DC001239D900DD1
:105690001124FC01E851FE4FFC8FEB8FADA1BEA1A0
:1056A0008D909D90AD90BC9020E030E0A901C501A7
:1056B000B4010E942D38882309F47FC02FA138A59A
:1056C00049A55AA5C501B4010E948F3A2B013C019E
:1056D000EDA1FEA160837183828393839B01AC0162
:1056E00060E070E080E89FE30E9437384B015C0186
:1056F000E894B7F8ADA5BEA51C962D913D914D91AE
:105700005C911F97C501B4010E948F3A6D8F7F8F06
:105710008C019B01AC0169A17AA18BA19CA10E9483
:105720002D3887FD06C0BD8DB9A3EF8DEAA30BA36D
:105730001CA3AB8DBC8DBC91BD8FEB8DFC8DF1811D
:10574000FF8FAB8DBC8D12960C91129713961C9106
:10575000EDA5FEA5208D318D428D538DC501B4017F
:105760000E948F3A4B015C019B01AC016D8D7F8DD6
:10577000C8010E942D3887FD03C08D8E9F8E850144
:105780008D8D9F8DD801EB8DFC8D80839183A283BD
:10579000B383ABA9BCA91C962D913D914D915C9111
:1057A0001F97C301B2010E948F3A9B01AC01C70150
:1057B000B6010E9437376B017C01EDA1FEA1349642
:1057C000FEA3EDA32BA93CA92C5F3F4F3CAB2BAB19
:1057D0004DA55EA54C5F5F4F5EA74DA7898D9A8D45
:1057E000E817F90709F05ACF9091AA048091A9040B
:1057F00098130DC089E2829DF001839DF00D112464
:10580000E953FE4F118A128A138A148A12C024EABD
:1058100030E74DE75FE3C701B6010E944F3A181623
:105820006CF489E2829DF001839DF00D1124E9530F
:10583000FE4F118E128E138E148E66C024EA30E74E
:105840004DE75FEBC701B6010E944F3A181644F0CE
:1058500084EAC82E80E7D82E8DE7E82E8FEBF82E4D
:10586000A701960160E070E080E89FE30E9437376F
:1058700020E030E040E05FE30E948F3A0E942E3B40
:105880006B017C0189E2829DF001839DF00D112462
:10589000E953FE4F20915D0630915E0640915F0610
:1058A0005091600661A172A183A194A10E948F3AD8
:1058B000A70196010E948F3A4B015C01A701960156
:1058C00060E070E080E89FE30E9437379B01AC0105
:1058D000C501B4010E9437386B017C0120E030E043
:1058E000A9010E942D3887FF03C0C12CD12C76015D
:1058F00089E2829DF001839DF00D1124E953FE4F52
:10590000C18ED28EE38EF48E29A13AA14BA15CA167
:1059100069A17AA18BA19CA10E948F3A7B018C0185
:1059200089E2829DF001839DF00D1124E953FE4F21
:10593000C701D801858F968FA78FB0A3A18CB28C99
:10594000C38CD48C60901B0170901C0180901D0151
:1059500090901E019301A401B701C8010E942D3847
:1059600087FD05C0762D672D982D892D04C07E2DCD
:105970006F2D902F812F272F362F492F582FB501AC
:10598000C6010E942D3887FD0DC09301A401B70107
:10599000C8010E942D3887FD03C05301640102C075
:1059A0005701680189E2829DF001839DF00D112469
:1059B000E953FE4FC501D601858B968BA78BB08F1F
:1059C0008CE0FE013196AFE0B1E001900D928A9536
:1059D000E1F7C701D80180931B0190931C01A093AC
:1059E0001D01B0931E018CE0FE013D96A3E0B1E0E5
:1059F00001900D928A95E1F7809102018093AA04AB
:105A00008F5F823109F480E080930201C75BDF4F32
:105A10000FB6F894DEBF0FBECDBFDF91CF911F91BF
:105A20000F91FF90EF90DF90CF90BF90AF909F903D
:105A30008F907F906F905F904F903F902F900C943D
:105A40003F04C75BDF4F0FB6F894DEBF0FBECDBF7C
:105A5000DF91CF911F910F91FF90EF90DF90CF904A
:105A6000BF90AF909F908F907F906F905F904F907E
:105A70003F902F900895CF93DF93CDB7DEB7619716
:105A80000FB6F894DEBF0FBECDBF8091C00082601C
:105A90008093C0001092C50080E18093C400809183
:105AA000C10080618093C1008091C10088608093B3
:105AB000C1008091C10080688093C10080E090E0C7
:105AC0000E942604893009F038C54FE450E061E0B7
:105AD00070E088E296E00E949505892B09F42DC5B7
:105AE0008AB18C618AB9209A8AB1806E8AB9809114
:105AF00081008F7E809381008091810088608093F7
:105B00008100809180008C7F809380008091800054
:105B10008F708093800080916E00887F80936E00EC
:105B200014BC15BC80916E00816080936E0087B1BB
:105B3000887F87B988B1876088B980916C00876059
:105B400080936C008091680082608093680080E29E
:105B5000E1EBF6E0DF011D928A95E9F781E08093A1
:105B6000B10678949091650694FD8093B20659EE43
:105B7000C52E55E0D52E662463948091A0018093B4
:105B80009F018FE3F60111928A95E9F76CE076E0C8
:105B900080E00E948825811103C087E00E94651380
:105BA000239A259A0E9409253B9A0E943C063D981B
:105BB000459A0E942E040E94A7220E94DD1766EBE0
:105BC00076E080E096E00E94EA181092B10610920A
:105BD000B4061092B5061092B30684E391E00E94D9
:105BE00056138091B206813099F48FEB93E00E94B6
:105BF000561389E993E00E9456138CE493E00E94C7
:105C0000561310E000E033E0732E42E0E42E21C092
:105C10001092B2060E946C18F4CFE92FF0E0E15E1A
:105C2000FE4F80819F5F903809F490E090939F0130
:105C30008F3FA9F08A30E1F4E12FF0E0E756FA4F08
:105C400010820E943D150091B1060023A9F010E0DA
:105C500000E090919F018091A0018913DECF0E9406
:105C600023130E943D158091B106882391F385CFBF
:105C70008D3009F036C4E0CF80919905811105C0BF
:105C800088E098E00E94561343C4843209F01CC493
:105C9000698A80919A05833481F034F4882351F025
:105CA000843209F019C109C0873439F0883509F008
:105CB00013C103C088E092E0D6C090919B0591117A
:105CC000FCC3833409F4D2C01CF4843239F0FAC323
:105CD000873471F0883509F4EBC0F4C38091B206C3
:105CE000082F087111F008E0EDC30E94D113EAC338
:105CF00086E092E00E9456138091E905823091F08F
:105D000038F4882361F08130A9F480E092E00CC07F
:105D1000833069F0883071F486EF91E005C083E04C
:105D200092E002C08DEF91E00E9456130CC08AEF02
:105D300091E0FACF81EF91E00E9456138091E9053E
:105D400086500E944A138EEE91E00E945613809175
:105D5000EF058A5C0E944A138091ED05813049F07D
:105D600028F0823051F48FED91E005C089EE91E08A
:105D700002C084EE91E00E9456138091EB058111E0
:105D800003C08AED91E002C085ED91E00E945613B8
:105D90008091EC05811103C080ED91E002C08BEC95
:105DA00091E00E9456138091EA05813019F486EC47
:105DB00091E002C081EC91E00E9456138091F005C1
:105DC000813049F028F0823051F485EB91E005C034
:105DD0008DEB91E002C089EB91E00E945613809117
:105DE000F205813031F040F0823051F48DEA91E0DB
:105DF00005C081EB91E002C089EA91E00E94561350
:105E00008091F105882329F0823039F481EA91E00C
:105E100002C085EA91E00E9456138EE991E00E944B
:105E200056138091FB050E944A138BE991E00E9472
:105E300056136091F7057091F8058091F9059091DE
:105E4000FA050E942C1388E991E00E945613609194
:105E5000F3057091F4058091F5059091F6050E9487
:105E60002C1384E991E00E9456132CC38091B20652
:105E7000823069F40E943E068FEB93E00E94561335
:105E800086E793E00E9456138CE493E0ECCF8111F7
:105E90002ACFE092B2068FEB93E00E9456138FE771
:105EA00093E00E9456138CE493E00E9456133BC08B
:105EB0008091B206813009F005C38FEB93E00E9418
:105EC000561387E893E00E9456138CE493E00E94F7
:105ED00056131092B206F6C29091B206923008F0B4
:105EE00002CF893409F4B1C034F4833259F08834D4
:105EF00009F483C04AC18E3409F41EC1823509F405
:105F0000E3C043C1E98A80919B058111D6C210E0AC
:105F1000BE016F5F7F4F812F0E948825811105C0D0
:105F200087E00E94651300E0CDC281E991E00E9404
:105F30005613163029F0173041F48BE891E002C077
:105F40008EE891E00E94561304C086E3810F0E9400
:105F50004A1389E891E00E945613CE0101965C0134
:105F6000F12CD5016D917D918D919D915D010E94E6
:105F70003B13B2E0FB1619F087E891E002C083E81A
:105F800091E00E945613F394E3E0FE12EACF1F5F04
:105F9000183009F0BDCF8DE791E00E94561328E13B
:105FA000A22E26E0B22E10E0D5016D917D918D914B
:105FB0009D915D010E943B13123019F08BE791E037
:105FC00002C087E791E00E9456131F5F133061F70C
:105FD00081E791E00E945613609124067091250696
:105FE00080912606909127060E943B138DE691E052
:105FF0000E9456130E94AE1365C28091650684FF0D
:1060000056C284E08093B20680916B00897E8093B3
:106010006B00809168008E7F809368000E943D1520
:106020008091B106811106C066EB76E080E096E0D3
:106030000E94EA188091B106811144C21092B20602
:106040000E947C220E946C186ECFE98A80919B0589
:1060500081111DC040E550E06EEA73E089E995E0EA
:106060000E949505892B51F41092990540E550E066
:1060700069E975E08EEA93E00E94FD058DE591E007
:106080000E9456130E94081289E591E0ECCE798AAD
:106090008D3309F012C283E0282F30E0F901E75672
:1060A000FA4F9081D901AA56BA4F9C938F5F908185
:1060B0009111F2CF898B40E550E069E975E08EEAF5
:1060C00093E00E94FD05FEC1E98A80919B0583351E
:1060D00009F0F3C1798A80919C05843509F0EDC1FE
:1060E00084E0898B80919D058D3309F0E6C1809114
:1060F0009F058111E2C185E0898B80919E058432E4
:1061000039F08A3239F0833209F0D7C182E003C016
:1061100081E001C08FEF0E94A9258FEB93E00E94E0
:10612000561380E593E00E9456138CE493E00E949E
:1061300056130E943E06C6C1E98A80919B058111D3
:1061400020C010E0812F0E941512811104C087E049
:106150000E94651311C086E591E00E945613812FBD
:106160000E944A1384E591E00E9456130E9408128F
:1061700081E591E00E945613113009F4A3C111E0AA
:10618000E1CF9111B0CD11E001C010E0BE01635F1D
:106190007F4FCE0141960E945D27811102C002E02F
:1061A00091C1E98981E08E0F898BF0E0E756FA4FC3
:1061B00090819D3309F081C1112359F1482F50E09E
:1061C000282F30E0D901A756BA4F9C91241B350BDC
:1061D000F901E756FA4F90838F5F9C919111F0CFB0
:1061E000898B0E949D06811164C16D857E858F8596
:1061F00098890E94723B0E94B038B1E56B9FC00144
:10620000112440E550E069E975E09D5F0E94FD05BD
:106210008ACEBE016F5F7F4FCE0141960E945D27FF
:10622000882309F4BCCFE989F0E0E756FA4F808172
:10623000811143C12D843E844F84588820E030E092
:106240004FE753E4C201B1010E944F3A18160CF413
:1062500034C189809A80AB80BC80C201B1010E94A8
:10626000B038162F20E030E0A901C501B4010E942A
:106270002D3887FD20C1143608F443C0145680E041
:106280001330B0F5212F30E0220F331F220F331FC0
:10629000F901823071F0833021F1813019F0E85D2D
:1062A000F94F02C0EC5CF94F80829182A282B382E6
:1062B000FBC0E05CF94F2F0120E030E040E752E402
:1062C000C501B4010E948F3A20E030E040E752E47B
:1062D0000E948F3AD2016D937D938D939C93139777
:1062E000E3C0E45BF94FB7FAB094B7F8B094DCCFF1
:1062F0008F5F1A3008F4E1C0843009F4DEC01A5010
:10630000BFCFC501B4010E94723B0E94B0381C305F
:1063100009F485C030F5143009F464C070F411300C
:1063200009F458C008F450C0123009F456C01330B4
:1063300009F0C3C060935A0652C0163009F464C015
:1063400008F45AC01A3009F467C01B3009F0B5C010
:1063500080925D0690925E06A0925F06B092600603
:10636000A3C0173109F486C078F4143109F468C069
:1063700020F41D3009F45CC0A0C0153109F46AC0D6
:10638000163109F46FC099C01A3109F47FC078F44E
:10639000183109F472C0193109F08FC080926D066E
:1063A00090926E06A0926F06B09270067DC01B316F
:1063B00009F472C0123409F080C0C501B4010E9412
:1063C000B03860936B0670C0633008F478C0609397
:1063D00058066AC060935B0667C0609359060E94C6
:1063E0004C2262C080916506662311F0846001C072
:1063F0008B7F8093650658C080916506662311F0F7
:106400008064F7CF8F7BF5CF80916506662311F00E
:106410008068EFCF8F77EDCF60935C0645C08092A8
:10642000610690926206A0926306B09264063CC038
:1064300080916506662311F08160DBCF8E7FD9CF16
:1064400080916506662321F084FF3BC08062D1CF36
:106450008F7DCFCF80916506662311F08860C9CF0C
:10646000877FC7CF80916506662311F08061C1CF19
:106470008F7CBFCF6093660617C0809267069092AC
:106480006806A0926906B0926A060EC070E070932A
:1064900072066093710608C080927306909274062B
:1064A000A0927506B09276060E9472250BC005E098
:1064B00009C0082F07C004E005C003E003C006E0E0
:1064C00001C00AE0802F0AC08091B206813021F419
:1064D00089E00E946513BBCB0E949D060E94351582
:1064E000B6CB002331F0893209F0B3CB013019F576
:1064F000AFCB813208F4ADCB8F3209F4AACB88320E
:10650000C1F08B33C1F01F3428F08BE00E9465137B
:1065100010E09FCB212F30E0E1E0E10F9FE9980FE1
:10652000D901A756BA4F9A3108F480528C931E2F86
:1065300090CB01E08ECB02E08CCB87E00E9465130C
:106540008FEF0E94A9250E94D113CACACF930E943F
:106550002313C9E20E943D158091B106811111C03B
:106560008091A9049091AA04981739F0C89FC0019E
:10657000112489539E4F892B69F78091B206883088
:1065800049F3CF910895CF92DF92EF92FF92CF938C
:10659000C82F6A017B0190916C068091B206913000
:1065A00009F053C0823009F466C00E9423130E9490
:1065B000A632C11103C00E9409253EC0C13011F4AA
:1065C0002D9801C02D9A83E88093B0008091B1008E
:1065D00087608093B10020E030E0A901C701B601D7
:1065E0000E942D3887FD11C020E030E044EB52E4DA
:1065F000C701B6010E944F3A181654F4C12CD12C91
:1066000084EBE82E82E4F82E03C0C12CD12C760155
:1066100027E13CE641E45EE3C701B6010E948F3A00
:1066200020E030E040E751E40E9438370E941C39F6
:106630000E94B0386093B30086E990E0CF91FF905C
:10664000EF90DF90CF900C948A058230A1F00E94E9
:10665000A63220E030E040E251E4C701B6010E94DA
:106660003738AB01BC018C2FCF91FF90EF90DF90BA
:10667000CF900C941725CF91FF90EF90DF90CF90A3
:106680000895FF920F931F93CF93DF9300D000D014
:10669000CDB7DEB73091B206323009F492C0F22E97
:1066A000142FAB01BC0149835A836B837C830E9406
:1066B000A6321092D0061092770680916506498125
:1066C0005A816B817C8187FD03C080E280937706CD
:1066D000FF2031F09091770680E28927809377063A
:1066E00086B1807290917706891791F09FB7F894E0
:1066F0008091B50680618093B5069FBF49835A8318
:106700006B837C830E943D157C816B815A8149811A
:106710008091B106811155C0212F85EA96E00E9433
:106720000E2881E08093C3069FB7F8948091B40649
:1067300082608093B4069FBF0E943D158091B10690
:1067400081113FC08091B2068111F6CF8091C306BE
:106750008130A9F4002351F08CE0E6EBF6E0A4ECE4
:10676000B6E001900D928A95E1F70CC09FB7F894BE
:106770008091B50680618093B5069FBF03C081E01C
:106780008093D0061092C3060E943D158091B106F9
:10679000811117C00E94A7220E942E040E94DD17BB
:1067A00066EB76E085EA96E00E94EA180F900F907B
:1067B0000F900F90DF91CF911F910F91FF900C944C
:1067C000AE130F900F900F900F90DF91CF911F910C
:1067D0000F91FF9008952F923F924F925F926F9288
:1067E0007F928F929F92AF92BF92CF92DF92EF9261
:1067F000FF920F931F93CF93DF93CDB7DEB7AF9781
:106800000FB6F894DEBF0FBECDBF69877A878B873E
:106810009C872B8B3C8B4D8B5E8B0F8BAD82898A3B
:1068200024E0E29E80011124C80180509A4F998F84
:10683000888FD801A957B94FBB8FAA8F8D909D9093
:10684000AD90BC90FC012081318142815381C50112
:10685000B4010E9438376C8F7D8F8E8F9F8FF4E04C
:10686000CF9E10011124910120503A4F39A328A343
:10687000C1018957994F9BA38AA3DC01CD90DD907C
:10688000ED90FC90F9012081318142815381C70153
:10689000B6010E9438376CA37DA38EA39FA3240169
:1068A000350177FA709477F87094D701C601B05823
:1068B00089839A83AB83BC83F801EB55F94F2C8D08
:1068C0003D8D4E8D5F8D60817181828193810E94AB
:1068D00037374B015C01F101EB55F94F2CA13DA17C
:1068E0004EA15FA160817181828193810E943737BF
:1068F0006B017C01A5019401C301B2010E948F3A92
:106900006D877E878F87988BA701960169817A8131
:106910008B819C810E948F3A9B01AC016D857E85A5
:106920008F8598890E9438376D877E878F87988BEF
:10693000A7019601C301B2010E948F3A6B017C014D
:10694000A501940169817A818B819C810E948F3A93
:106950009B01AC01C701B6010E9437372D853E85EA
:106960004F8558890E94B7376B017C01998999231B
:1069700099F02DEB37E346E055EBC701B6010E94D5
:106980004F3A87FD1DC02BED3FE049EC50E4C701B5
:10699000B6010E94373712C02DEB37E346E055E3CE
:1069A000C701B6010E942D38181654F02BED3FE0B8
:1069B00049EC50E4C701B6010E9438376B017C01F5
:1069C0008090610690906206A0906306B090640685
:1069D00029853A854B855C85CA01B9010E94383703
:1069E000A50194010E9437379B01AC01C501B40198
:1069F0000E948F3A0E942E3B4B015C0120E030E068
:106A000040E05FE3C701B6010E948F3A29853A85CD
:106A10004B855C850E948F3A9F77A50194010E9467
:106A200037380E941C390E94B0388B0161157105FE
:106A300009F476C14B01A12CB12CAF89AA2381F0B6
:106A4000C501B4010E94DF389B01AC016B897C89D0
:106A50008D899E890E948F3A6B8B7C8B8D8B9E8B50
:106A6000C501B4010E94DF384B015C019B01AC0100
:106A7000C701B6010E94373869877A878B879C8760
:106A8000ED81B4E0EB9FC00111249C0120503A4FEE
:106A90003A8B298BFC01EB55F94FD9012D913D9192
:106AA0004D915C9160817181828193810E94373721
:106AB000A50194010E9437386CA77DA78EA79FA7D8
:106AC00029853A854B855C85CA01B9010E948F3AB8
:106AD0009B01AC0160E070E080E090E40E943737F9
:106AE0006B017C012BEA3AEA4AE25EE369857A852A
:106AF0008B859C850E948F3A4B015C0120E030E041
:106B000040E850E4C701B6010E9438379B01AC0150
:106B1000C501B4010E948F3A6D877E878F87988B5D
:106B200020E030E040E05FE3C701B6010E948F3A09
:106B300068A779A78AA79BA71D8222242394312CBA
:106B40002016310609F4ECC0BD81BC3008F040C00D
:106B500028A539A54AA55BA569817A818B819C818D
:106B60000E948F3A6B017C012D853E854F855889A7
:106B7000C301B2010E948F3AA70196010E943837E3
:106B80007B016C0128A539A54AA55BA5C301B2010B
:106B90000E948F3A4B015C012D853E854F855889B7
:106BA00069817A818B819C810E948F3A9B01AC0123
:106BB000C501B4010E9437372B013C01ED81EF5F25
:106BC000ED83C701D60189839A83AB83BC8365C0FB
:106BD000B10180E090E00E94DF3829853A854B853D
:106BE0005C850E948F3A6B017C010E943238698378
:106BF0007A838B839C83C701B6010E94203B4B01A3
:106C00005C01AA8DBB8DCD90DD90ED90FC90F7FAE4
:106C1000F094F7F8F094AAA1BBA18D919D910D90ED
:106C2000BC91A02D8D839E83AF83B88729813A8143
:106C30004B815C81C701B6010E948F3A2B013C0158
:106C4000A50194016D817E818F8198850E948F3A84
:106C50009B01AC01C301B2010E9438372B013C01FA
:106C6000A5019401C701B6010E948F3A6B017C0116
:106C700029813A814B815C816D817E818F819885EC
:106C80000E948F3A9B01AC01C701B6010E943737C1
:106C900069837A838B839C831D82A30192016C8D0F
:106CA0007D8D8E8D9F8D0E943837E88DF98D6083A4
:106CB00071838283938329813A814B815C816CA1AA
:106CC0007DA18EA19FA10E943837A8A1B9A16D9383
:106CD0007D938D939C9313972CA53DA54EA55FA501
:106CE000E989FA8960817181828193810E943837B4
:106CF000A989BA896D937D938D939C9313972F895E
:106D00004B895C896D897E8980E096E00E940E281F
:106D10008091B106811125C0BFEF2B1A3B0A10CF1D
:106D20002F894B895C896D897E8985EA96E0AF96CB
:106D30000FB6F894DEBF0FBECDBFDF91CF911F918C
:106D40000F91FF90EF90DF90CF90BF90AF909F900A
:106D50008F907F906F905F904F903F902F900C940A
:106D60000E28AF960FB6F894DEBF0FBECDBFDF91F1
:106D7000CF911F910F91FF90EF90DF90CF90BF9038
:106D8000AF909F908F907F906F905F904F903F90CB
:106D90002F900895991B79E004C0991F961708F069
:106DA000961B881F7A95C9F780950895A1E21A2E3F
:106DB000AA1BBB1BFD010DC0AA1FBB1FEE1FFF1F9F
:106DC000A217B307E407F50720F0A21BB30BE40BEF
:106DD000F50B661F771F881F991F1A9469F7609536
:106DE0007095809590959B01AC01BD01CF010895F0
:106DF000052E97FB1EF400940E940F3757FD07D015
:106E00000E94D63607FC03D04EF40C940F375095F1
:106E10004095309521953F4F4F4F5F4F0895909586
:106E20008095709561957F4F8F4F9F4F0895EE0F1E
:106E3000FF1F0590F491E02D09940E942837A59F2B
:106E4000900DB49F900DA49F800D911D1124089565
:106E5000A29FB001B39FC001A39F700D811D11249B
:106E6000911DB29F700D811D1124911D08955058E0
:106E7000BB27AA270E944F370C94E9390E94B039EA
:106E800038F00E94B73920F039F49F3F19F426F406
:106E90000C9486390EF4E095E7FB0C945739E92FF2
:106EA0000E940E3A58F3BA176207730784079507D2
:106EB00020F079F4A6F50C94483A0EF4E0950B2EE8
:106EC000BA2FA02D0B01B90190010C01CA01A0013C
:106ED0001124FF27591B99F0593F50F4503E68F197
:106EE0001A16F040A22F232F342F4427585FF3CFD8
:106EF000469537952795A795F0405395C9F77EF4A9
:106F00001F16BA0B620B730B840BBAF09150A1F0F1
:106F1000FF0FBB1F661F771F881FC2F70EC0BA0F77
:106F2000621F731F841F48F4879577956795B795FF
:106F3000F7959E3F08F0B0CF9395880F08F09927FA
:106F4000EE0F9795879508950E94B03960F080E81C
:106F500091E009F49EEF0E94B73928F040E851E033
:106F600071F45EEF0CC00C9486390C94483AE92F0A
:106F7000E0780E940E3A40F3092E052AB1F3261755
:106F800037074807590738F00E2E07F8E02569F053
:106F9000E025E0640AC0EF6307F8009407FADB011C
:106FA000B9019D01DC01CA01AD01EF930E944E3889
:106FB0000E94E9390E94E7375F91552339F02BEDA4
:106FC0003FE049E450FD49EC0C9438370895DF93D5
:106FD000DD27B92FBF7740E85FE31616170648078D
:106FE0005B0718F4D92F0E94543A9F938F937F9395
:106FF0006F930E946E3BE8EEF0E00E9489390E9498
:10700000E9392F913F914F915F910E94A23ADD2380
:1070100051F09058A2EA2AED3FE049EC5FE3D078C6
:107020005D270E944F37DF910C94E9390E94303A76
:1070300090F09F3748F4911116F40C94493A60E0AF
:1070400070E080E89FE3089526F01B16611D711D16
:10705000811D0C945D390C9478390E94333908F401
:1070600081E008950E94C039E3950C94FA390E949A
:107070004B380C94E9390E94B73958F00E94B03966
:1070800040F029F45F3F29F00C94573951110C94CA
:10709000493A0C9486390E940E3A68F39923B1F369
:1070A000552391F3951B550BBB27AA27621773072E
:1070B000840738F09F5F5F4F220F331F441FAA1FC2
:1070C000A9F335D00E2E3AF0E0E832D0915050407E
:1070D000E695001CCAF72BD0FE2F29D0660F771F2C
:1070E000881FBB1F261737074807AB07B0E809F012
:1070F000BB0B802DBF01FF2793585F4F3AF09E3F97
:10710000510578F00C9457390C94493A5F3FE4F3F9
:10711000983ED4F3869577956795B795F7959F5FD9
:10712000C9F7880F911D9695879597F90895E1E025
:10713000660F771F881FBB1F621773078407BA0784
:1071400020F0621B730B840BBA0BEE1F88F7E095DF
:1071500008950E94B0386894B1110C94493A08958A
:107160000E94163A88F09F5798F0B92F9927B75187
:10717000B0F0E1F0660F771F881F991F1AF0BA95DB
:10718000C9F714C0B13091F00E94483AB1E00895B7
:107190000C94483A672F782F8827B85F39F0B93FA9
:1071A000CCF3869577956795B395D9F73EF490958E
:1071B0008095709561957F4F8F4F9F4F0895E8940C
:1071C00009C097FB3EF490958095709561957F4F2F
:1071D0008F4F9F4F9923A9F0F92F96E9BB279395DD
:1071E000F695879577956795B795F111F8CFFAF4ED
:1071F000BB0F11F460FF1BC06F5F7F4F8F4F9F4F1E
:1072000016C0882311F096E911C0772321F09EE87B
:10721000872F762F05C0662371F096E8862F70E0E1
:1072200060E02AF09A95660F771F881FDAF7880FBB
:107230009695879597F908950E94303A90F09F3778
:1072400048F4911116F00C94493A60E070E080E83F
:107250009FEB089526F41B16611D711D811D0C9472
:107260005D390C947839990F0008550FAA0BE0E8A6
:10727000FEEF16161706E807F907C0F012161306F8
:10728000E407F50798F0621B730B840B950B39F438
:107290000A2661F0232B242B252B21F408950A269E
:1072A00009F4A140A6958FEF811D811D089597F9DE
:1072B0009F6780E870E060E00895882371F4772389
:1072C00021F09850872B762F07C0662311F4992759
:1072D0000DC09051862B70E060E02AF09A95660F01
:1072E000771F881FDAF7880F9695879597F9089585
:1072F0009F3F31F0915020F4879577956795B7952A
:10730000880F911D9695879597F908959FEF80ECCA
:107310000895DF93CF931F930F93FF92EF92DF9225
:107320007B018C01689406C0DA2EEF010E94A23A1C
:10733000FE01E894A5912591359145915591A6F3CB
:10734000EF010E944F37FE019701A801DA9469F717
:10735000DF90EF90FF900F911F91CF91DF910895F3
:1073600000240A9416161706180609060895002424
:107370000A94121613061406050608950C9486390D
:107380000E94163AD8F3E894E0E0BB279F57F0F04C
:107390002AED3FE049EC06C0EE0FBB0F661F771FDA
:1073A000881F28F0B23A62077307840728F0B25AA0
:1073B000620B730B840BE3959A9572F7803830F467
:1073C0009A95BB0F661F771F881FD2F790480C94C1
:1073D0007A39092E0394000C11F4882352F0BB0F64
:1073E00040F4BF2B11F460FF04C06F5F7F4F8F4FDD
:1073F0009F4F0895EF93E0FF07C0A2EA2AED3FE018
:1074000049EC5FEB0E944F370E94E9390F900394DB
:1074100001FC9058E5E1F1E00C94843B57FD905855
:10742000440F551F59F05F3F71F04795880F97FB48
:10743000991F61F09F3F79F0879508951216130602
:107440001406551FF2CF4695F1DF08C01616170631
:107450001806991FF1CF8695710561050894089566
:107460000E94163AA0F0BEE7B91788F4BB279F38F0
:1074700060F41616B11D672F782F8827985FF7CF15
:10748000869577956795B11D93959639C8F30895BC
:10749000E894BB2766277727CB0197F908950E94C8
:1074A000333908F48FEF08959B01AC0160E070E080
:1074B00080E89FE30C9437380E94163A58F19E57A3
:1074C00060F19851A0F0E9F0983020F5092E992745
:1074D000660F771F881F991F0A94D1F712C0062ED6
:1074E000672F782F8827985F11F4000C07C0993F09
:1074F000B4F38695779567959395D9F7611D711DBE
:10750000811D3EF490958095709561957F4F8F4FCA
:107510009F4F089568940C94493A0C94483A0E94FD
:10752000A23A0C94E9390E94B03938F00E94B73978
:1075300020F0952311F00C9457390C9486391124BE
:107540000C94493A0E940E3A70F3959FC1F3950F3F
:1075500050E0551F629FF001729FBB27F00DB11DD7
:10756000639FAA27F00DB11DAA1F649F6627B00D67
:10757000A11D661F829F2227B00DA11D621F739F50
:10758000B00DA11D621F839FA00D611D221F749F5E
:107590003327A00D611D231F849F600D211D822FA5
:1075A000762F6A2F11249F5750409AF0F1F08823CC
:1075B0004AF0EE0FFF1FBB1F661F771F881F9150F9
:1075C0005040A9F79E3F510580F00C9457390C9418
:1075D000493A5F3FE4F3983ED4F3869577956795F3
:1075E000B795F795E7959F5FC1F7FE2B880F911D23
:1075F0009695879597F908950E94163AE8F09E3778
:10760000E8F09639B8F49E3848F4672F782F882729
:10761000985FF9CF86957795679593959539D0F3CF
:10762000B62FB1706B0F711D811D20F48795779572
:10763000679593950C945D390C9478390C94493A7C
:107640009F930E94C0390F9007FCEE5F0C94FA39AB
:1076500019F416F40C9486390C9478390E94163A71
:10766000B8F39923C9F3B6F39F57550B87FF0E94D0
:107670007D3B0024A0E640EA9001805856959795FE
:1076800028F4805C660F771F881F20F026173707C5
:10769000480730F4621B730B840B202931294A2BD5
:1076A000A69517940794202531254A2758F7660F89
:1076B000771F881F20F026173707480730F4620B22
:1076C000730B840B200D311D411DA09581F7B9016D
:1076D000842F9158880F9695879508959B01AC014A
:1076E0000C948F3A0E94303A30F09F3710F40C948B
:1076F000493A0C945D390C94783991505040660F9A
:10770000771F881FD2F708959F938F937F936F936E
:10771000FF93EF939B01AC010E948F3AEF91FF9191
:107720000E9489392F913F914F915F910C948F3A2C
:04773000F894FFCFFB
:02773400010052
:00000001FF
